:020000040000FA
:06000000D6EF32F0120001
:0600080039EF2FF0120099
:0600180018EF2FF01200AA
:06002A000400E265000085
:100030000901000008000000E16500002101000046
:1000400001000000DE6500001C010000030000004C
:0C005000DA65000015010000040000004B
:04005C000001010E90
:10006000CD6FE66ECFEC17F0E55212000001020EE4
:10007000CD6FE66ECFEC17F0E55212000001030ED3
:10008000CD6FE66ECFEC17F0E55212000001020EC4
:10009000CC6FCCC0E6FF35EC20F0E5521200000139
:1000A000CC0502E0000E01D0010E00D01200D9CF25
:1000B000E6FFE1CFD9FF0F0EE126010EDB6ADF6A12
:1000C0000C0EDF5C11E2DF50080DF3CFE9FFF4CF37
:1000D000EAFF600EE926000EEA22070EE926000E6E
:1000E000EA22EF6ADF2AECD7DF6A040EDF5C09E25E
:1000F000DF50EA6AC00FE96E000EEA22EF6ADF2ADB
:10010000F4D70001D06B74EC2FF0F3CFCEF0F4CF26
:10011000CFF0FE0EDB5003E0FE0EDB040EE1070E17
:10012000E66EBF0EE66E430EE66E82EC17F0E55209
:10013000E552E552DE52010EDD6EFE0EDB5001E0AF
:1001400078D094DF020EF36EFE0EF3CFDBFFD950B2
:10015000060FE66E000EDA20E66ED950070FE66E47
:10016000000EDA20E66ED950020FE66E000EDA209D
:10017000E66EEFEC24F0F56E060EE15EF550000938
:1001800031E1D950020FE96EDACFEAFFEF0EEE1837
:1001900006E1070EEE1803E1EE5001E1EE5022E118
:1001A000060EDB5008081EE1080EE66EE66ADC0E5D
:1001B000E66E600EE66ED950070FE66E000EDA208E
:1001C000E66ED5EC2FF0F56E060EE15EF5500009F7
:1001D00009E1010EF36EFE0EF3CFDBFF0001010E0D
:1001E000D06F27D074EC2FF00001CE51F35C006E7D
:1001F000CF51F458016E00C0E6FF01C0E6FFC80E03
:10020000E66EE66A7AEC2FF0E552E552E552E7CF6A
:1002100001F0E552E7CF00F0F3CF02F0F4CF03F0A6
:100220000050025C0150035801E203D0D3EC2FF0E0
:100230008ED7FE0EDB5002082DE1C40EE66E000ED6
:10024000E66EACEC1EF0E552E552000908E0C40E83
:10025000E66E000EE66E3BEC1EF0E552E552010E36
:10026000DB500CE1CBC0E6FFCAC0E6FFC9C0E6FF29
:1002700082EC17F0E552E552E5520BD0CBC0E6FF19
:10028000CAC0E6FFC9C0E6FFB2EC17F0E552E5527E
:10029000E55208D0C40EE66E000EE66E3BEC1EF092
:1002A000E552E552010EE66EE66A59EC13F0E552AE
:1002B000E552FE0EDB50020802E1F5EC13F0D6DE4B
:1002C000A2EC12F0E3DEFE0EDB0402E0000E01D031
:1002D000010E006E016A00BE016800C0F3FF01C09C
:1002E000F4FF00D0D9CFE1FFE552E7CFD9FF1200EC
:1002F000D9CFE6FFE1CFD9FF020EE126F40EDBCF26
:10030000E6FFD950F90FE96EFF0EDA20EA6EEECF64
:10031000E6FFEECFE6FFEECFE6FFEFCFE6FF010E02
:10032000E66EFD0EDBCFE6FFFE0EDBCFE6FF6FECE9
:1003300006F0F56E080EE15EF550F3CFDEFFF4CF68
:10034000DDFFDECF00F0DDCF01F00001800E0114F3
:1003500004E0010EF36EF46A7DD0F70EDB5013E07B
:10036000DECFE9FFDDCFEAFF030ED890E936EA36AB
:10037000E806FBE1600EE926000EEA22070EE926F8
:10038000000EEA22EF82F60EDB5013E0DECFE9FF2B
:10039000DDCFEAFF030ED890E936EA36E806FBE146
:1003A000600EE926000EEA22070EE926000EEA2278
:1003B000EF84F50EDB5013E0DECFE9FFDDCFEAFF7F
:1003C000030ED890E936EA36E806FBE1600EE9262E
:1003D000000EEA22070EE926000EEA22EF86F80E4A
:1003E000DB50080828E3DECFE9FFDDCFEAFF030E8C
:1003F000D890E936EA36E806FBE1600EE926000E01
:10040000EA22050EE926000EEA22F80EDBCFEFFF06
:10041000DECFE9FFDDCFEAFF030ED890E936EA36FA
:10042000E806FBE1600EE926000EEA22070EE92647
:10043000000EEA22EF8ADECFE6FFDDCFE6FF84EC96
:1004400007F0E552E552F3CFDEFFF4CFDDFFF36AAC
:10045000F46A00D0D9CFE1FFE552E7CFD9FF12000F
:10046000D9CFE6FFE1CFD9FF0E0EE126D950040F18
:10047000E66E000EDA20E66ED950050FE66E000E2D
:10048000DA20E66ED9CFE6FFDACFE6FFE0EC17F030
:10049000F56E060EE15EF550E76E0D0EE7CFDBFF61
:1004A000DB5001E01BD0040EDBCFE6FFD950050F77
:1004B000E66E000EDA20E66ED9CFE9FFDACFEAFF6A
:1004C000EECFE6FFEECFE6FFEECFE6FFEFCFE6FFA3
:1004D0000BD8F56E070EE15EF550C8D7D9CFE1FF16
:1004E000E552E7CFD9FF1200D9CFE6FFE1CFD9FF20
:1004F000030EE1260001010ED06F006A016A026A54
:10050000400E036ED950FB0FE96EFF0EDA20EA6E43
:10051000EE500016EE500116EE500216EE50031685
:10052000005001100210031001E1B8D0006A016A06
:10053000026A800E036ED950FB0FE96EFF0EDA20BF
:10054000EA6EEE500016EE500116EE500216EE5016
:100550000316005001100210031002E1000E01D03A
:10056000010EE66ED950FB0FE96EFF0EDA20EA6E3F
:10057000EECFE6FFEECFE6FFEECFE6FFEFCFE6FFF2
:1005800011DBF56E050EE15EF550F3CFDEFFF4CF23
:10059000DDFFDECF00F0DDCF01F00001800E0114A1
:1005A0005FE1DECFE9FFDDCFEAFF030ED890E93649
:1005B000EA36E806FBE1600EE926000EEA22070EA5
:1005C000E926000EEA22EF50020B4AE0DECFE9FFF7
:1005D000DDCFEAFF030ED890E936EA36E806FBE104
:1005E000600EE926000EEA22040EE926000EEA2239
:1005F000EF0405E1E66A1BEC09F0E55230D000019A
:10060000CC052DE1DECFE9FFDDCFEAFF030ED89068
:10061000E936EA36E806FBE1600EE926000EEA223A
:10062000070EE926000EEA22EF50040BE66EDECF3D
:10063000E9FFDDCFEAFF030ED890E936EA36E80697
:10064000FBE1600EE926000EEA22040EE926000E08
:10065000EA22EF50E66E27EC23F0E552E5521DD07A
:10066000F90EDBCFE6FFFA0EDBCFE6FFF80EDBCFAD
:10067000E6FFD950FB0FE96EFF0EDA20EA6EEECFEF
:10068000E6FFEECFE6FFEECFE6FFEFCFE6FF2FEC83
:1006900023F0F56E070EE15EF550BFD0E66A006A02
:1006A000016A026A800E036ED950FB0FE96EFF0EDD
:1006B000DA20EA6EEE500016EE500116EE500216E9
:1006C000EE500316005001100210031002E1000E5C
:1006D00001D0010EE66ED950FB0FE96EFF0EDA2055
:1006E000EA6EEECFE6FFEECFE6FFEECFE6FFEFCF0E
:1006F000E6FFF6D9F56E060EE15EF550F3CFDEFFAC
:10070000F4CFDDFFDECF00F0DDCF01F00001800E81
:10071000011466E1DECFE9FFDDCFEAFF030ED890DA
:10072000E936EA36E806FBE1600EE926000EEA2229
:10073000070EE926000EEA22EF50020B51E0DECF51
:10074000E9FFDDCFEAFF030ED890E936EA36E80686
:10075000FBE1600EE926000EEA22040EE926000EF7
:10076000EA22020EEFCFDBFFDB500EE1F80EDBCF0B
:10077000E6FFF90EDBCFE6FFFA0EDBCFE6FF53D83C
:10078000E552E552E5522BD00001CC0513E1F80EFD
:10079000DBCFE6FFF90EDBCFE6FFFA0EDBCFE6FF9D
:1007A000020EDBCFE6FF3DEC20F0E552E552E552CC
:1007B000E55215D0020ECC5D12E1F80EDBCFE6FF5C
:1007C000F90EDBCFE6FFFA0EDBCFE6FF020EDBCF42
:1007D000E6FF0AEC23F0E552E552E552E5521DD062
:1007E000F90EDBCFE6FFFA0EDBCFE6FFF80EDBCF2C
:1007F000E6FFD950FB0FE96EFF0EDA20EA6EEECF6E
:10080000E6FFEECFE6FFEECFE6FFEFCFE6FF2FEC01
:1008100023F0F56E070EE15EF550D9CFE1FFE5520A
:10082000E7CFD9FF1200D9CFE6FFE1CFD9FF040E01
:10083000E126FD0EDBCFE9FFFE0EDBCFEAFFEFCFB7
:10084000DFFF010EE76EFD0EDBCFE9FFFE0EDBCF13
:10085000EAFFE750E926000EEA22010EEFCFDBFFA8
:10086000FC0EDB50080801E0BCD0DF5044E0000182
:10087000C851DF5C40E0020EDB6A030EDB6A020E49
:10088000DBCF00F0030EDBCF01F0D890015004E67F
:10089000040E005C000E015823E2020EDBCFE9FFDC
:1008A000030EDBCFEAFFC00EE926000EEA22EF506E
:1008B00001E197D0020EDBCFE9FF030EDBCFEAFFA9
:1008C000C00EE926000EEA22EFCF00F0DF50005CF8
:1008D00001E106D0020EDB2A030E01E3DB2ACFD7AB
:1008E000D950020FE96EDACFEAFF040EEE1801E1EB
:1008F000ED5001E176D0010EDB50810A67E0910AEC
:100900005AE0190A4DE0010A40E00C0A33E0070AF8
:1009100026E0010A19E0030A0DE0010A01E061D0B6
:10092000FD0EDBCFE6FFFE0EDBCFE6FF3BDBE55245
:10093000E55257D0FD0EDBCFE6FFFE0EDBCFE6FF24
:1009400085DBE552E5524DD0FD0EDBCFE6FFFE0E16
:10095000DBCFE6FFBFEC09F0E552E55242D0FD0ED9
:10096000DBCFE6FFFE0EDBCFE6FF4AEC0DF0E552F3
:10097000E55237D0FD0EDBCFE6FFFE0EDBCFE6FF04
:10098000CCEC0DF0E552E5522CD0FD0EDBCFE6FFAE
:10099000FE0EDBCFE6FFD1EC0EF0E552E55221D0A2
:1009A000FD0EDBCFE6FFFE0EDBCFE6FF13EC0FF014
:1009B000E552E55216D0FD0EDBCFE6FFFE0EDBCF93
:1009C000E6FF4AEC0FF0E552E5520BD0FD0EDBCF0F
:1009D000E6FFFE0EDBCFE6FFC1EC11F0E552E5527B
:1009E00000D0D9CFE1FFE552E7CFD9FF1200D9CF30
:1009F000E6FFE1CFD9FFE652FD0EDB5035E0DF6ABE
:100A00000C0EDF5C30E2DF50080DF3CFE9FFF4CFCE
:100A1000EAFF600EE926000EEA22040EE926000E27
:100A2000EA22EFCF00F0FE0EDB50005C1AE1DF504F
:100A3000080DF3CFE9FFF4CFEAFF600EE926000EC0
:100A4000EA22070EE926000EEA22EF50050B050800
:100A500008E1DF50006E016A00C0F3FF01C0F4FF3F
:100A60003AD0DF2ACDD734D0DF6A0C0EDF5C30E21B
:100A7000DF50080DF3CFE9FFF4CFEAFF600EE9265F
:100A8000000EEA22040EE926000EEA22EFCF00F063
:100A9000FE0EDB50005C1AE1DF50080DF3CFE9FFDA
:100AA000F4CFEAFF600EE926000EEA22070EE926DF
:100AB000000EEA22EF50050B010808E1DF50006E3E
:100AC000016A00C0F3FF01C0F4FF05D0DF2ACDD7D3
:100AD000F368F46800D0E552E552E7CFD9FF120081
:100AE000D9CFE6FFE1CFD9FF020EE126DE52010E9B
:100AF000DD6EFA0EDB5002E0010EDB88F90EDB50F2
:100B000002E0010EDB84DF6A0C0EDF5C42E2FB0ECA
:100B1000DBCF00F0FC0EDBCF01F0FD0EDBCF02F0EF
:100B2000FE0EDBCF03F0DF50080DF3CFE9FFF4CF6B
:100B3000EAFF600EE926000EEA22EE50001809E1F5
:100B4000EE50011806E1EE50021803E1EE500318D2
:100B500000E11DE1DF50080DF3CFE9FFF4CFEAFF1C
:100B6000600EE926000EEA22070EE926000EEA22B0
:100B7000EF50150B046E010EDB50045C08E1DF50F2
:100B8000006E016A00C0F3FF01C0F4FF05D0DF2A48
:100B9000BBD7F368F46800D0D9CFE1FFE552E7CFC7
:100BA000D9FF1200D9CFE6FFE1CFD9FF020EE1262F
:100BB000DE52090EDD6EFA0EDB5002E0010EDB881C
:100BC000DF6A0C0EDF5C42E2FB0EDBCF00F0FC0EB6
:100BD000DBCF01F0FD0EDBCF02F0FE0EDBCF03F02A
:100BE000DF50080DF3CFE9FFF4CFEAFF600EE926EE
:100BF000000EEA22EE50001809E1EE50011806E15D
:100C0000EE50021803E1EE50031800E11DE1DF5041
:100C1000080DF3CFE9FFF4CFEAFF600EE926000EDE
:100C2000EA22070EE926000EEA22EF50190B046EA5
:100C3000010EDB50045C08E1DF50006E016A00C069
:100C4000F3FF01C0F4FF05D0DF2ABBD7F368F468D7
:100C500000D0D9CFE1FFE552E7CFD9FF1200D9CFBD
:100C6000E6FFE1CFD9FFE652DF6A0C0EDF5C2FE230
:100C7000DF50080DF3CFE9FFF4CFEAFF600EE9265D
:100C8000000EEA22060EE926000EEA22EFCF00F05F
:100C9000FE0EDB50005C19E1DF50080DF3CFE9FFD9
:100CA000F4CFEAFF600EE926000EEA22070EE926DD
:100CB000000EEA22EF50010B08E0DF50006E016ADF
:100CC00000C0F3FF01C0F4FF05D0DF2ACED7F368E0
:100CD000F46800D0E552E552E7CFD9FF1200D9CF32
:100CE000E6FFE1CFD9FF060EE126020EDB68030E18
:100CF000DB68040EDB68050EDB680B0EDE6EDD6A5A
:100D0000DECF00F0DDCF01F00001800E011448E1DC
:100D1000DECFE9FFDDCFEAFF030ED890E936EA36F1
:100D2000E806FBE1600EE926000EEA22070EE9263E
:100D3000000EEA22EF50010B24E0DECFE9FFDDCF09
:100D4000EAFF030ED890E936EA36E806FBE1600ECA
:100D5000E926000EEA22060EE926000EEA22EFCF6F
:100D600000F0FE0EDB50005C0BE1D9CFE9FFDACFDB
:100D7000EAFF020EEECFDBFF030EEDCFDBFF10D05C
:100D80000AD0D9CFE9FFDACFEAFF040EEECFDBFFBE
:100D9000050EEDCFDBFFDF06010E01E2DB06B0D76B
:100DA000020EDBCF00F0030EDBCF01F00001800E5E
:100DB000011406E1020EDBCFDEFFDBCFDDFF11D039
:100DC000040EDBCF00F0050EDBCF01F0800E011426
:100DD00003E0F368F46892D0040EDBCFDEFFDBCFD4
:100DE000DDFFDECFE9FFDDCFEAFF030ED890E93665
:100DF000EA36E806FBE1600EE926000EEA22060E5E
:100E0000E926000EEA22FE0EDBCFEFFFDECFE9FF80
:100E1000DDCFEAFF030ED890E936EA36E806FBE1BB
:100E2000600EE926000EEA22040EE926000EEA22F0
:100E3000FD0EDBCFEFFFDECFE9FFDDCFEAFF030ED4
:100E4000D890E936EA36E806FBE1600EE926000EA6
:100E5000EA22F80EDBCFEEFFF90EDBCFEEFFFA0E43
:100E6000DBCFEEFFFB0EDBCFEEFFDECFE9FFDDCF0A
:100E7000EAFF030ED890E936EA36E806FBE1600E99
:100E8000E926000EEA22070EE926000EEA22010EEC
:100E9000EF6EFC0EDB5013E0DECFE9FFDDCFEAFFA3
:100EA000030ED890E936EA36E806FBE1600EE92643
:100EB000000EEA22070EE926000EEA22EF8CF70E5A
:100EC000DB5013E0DECFE9FFDDCFEAFF030ED89061
:100ED000E936EA36E806FBE1600EE926000EEA2272
:100EE000070EE926000EEA22EF88DECF00F0DDCF04
:100EF00001F000C0F3FF01C0F4FF00D0D9CFE1FF43
:100F0000E552E7CFD9FF1200D9CFE6FFE1CFD9FFF5
:100F1000FD0EDBCF00F0FE0EDBCF01F000C0F3FFD3
:100F200001C0F4FF00D0E552E7CFD9FF1200D9CFBE
:100F3000E6FFE1CFD9FFFD0EDBCF00F0FE0EDBCFE9
:100F400001F00001800E011429E1FD0EDBCFE9FF65
:100F5000FE0EDBCFEAFF030ED890E936EA36E8064C
:100F6000FBE1600EE926000EEA22070EE926000EDC
:100F7000EA22EF6AFD0EDBCFE9FFFE0EDBCFEAFFD0
:100F8000030ED890E936EA36E806FBE1600EE92662
:100F9000000EEA22EE68EE68EE68EE68E552E7CFF2
:100FA000D9FF1200D9CFE6FFE1CFD9FF020EE1262B
:100FB000E76EFD0EDBCFE9FFFE0EDBCFEAFFE75069
:100FC000E926000EEA22EF50030BDF6E030EE76EF8
:100FD000FD0EDBCFE9FFFE0EDBCFEAFFE750E9268F
:100FE000000EEA22EF50030BE76E010EE7CFDBFFA6
:100FF000DF500EE0DFCFCCF0030E0001CC5D03E14B
:10100000D4EC2FF005D0CCC0E6FF35EC20F0E55253
:10101000010EDB5015E0010EDBCFCDF0DB0403E168
:101020002EEC00F00DD0010EDB50020803E136EC8F
:1010300000F006D0010EDB50030802E13EEC00F0A8
:10104000D9CFE1FFE552E7CFD9FF1200D9CFE6FFB4
:10105000E1CFD9FF040EE126E76EFD0EDBCFE9FFFD
:10106000FE0EDBCFEAFFE750E926000EEA22EFCFC3
:1010700000F0016A026A036A050EE76EFD0EDBCF1F
:10108000E9FFFE0EDBCFEAFFE750E926000EEA2279
:10109000EFCF04F0056A066A076A080E1F0B07E027
:1010A000D8900436053606360736E806F9E10450CE
:1010B0000026055001220650022207500322060E88
:1010C000E76EFD0EDBCFE9FFFE0EDBCFEAFFE75058
:1010D000E926000EEA22EFCF08F0096A0A6A0B6AD5
:1010E000100E1F0B07E0D890083609360A360B366B
:1010F000E806F9E108500026095001220A500222B0
:101100000B500322070EE76EFD0EDBCFE9FFFE0E4C
:10111000DBCFEAFFE750E926000EEA22EF501F0B73
:101120000C6E0D6A0E6A0F6A180E1F0B07E0D8903E
:101130000C360D360E360F36E806F9E10C50002657
:101140000D5001220E5002220F50032200C0DFFF7B
:10115000010E01C0DBFF020E02C0DBFF030E03C065
:10116000DBFFD9CFE9FFDACFEAFFEECF00F0EECF19
:1011700001F0EECF02F0EFCF03F0005001100210AB
:10118000031034E0D9CFE9FFDACFEAFFE868EE18C0
:1011900008E1E868EE1805E1E868EE1802E11F0EC4
:1011A000EE1806E10001C469C569C669C7691CD0AB
:1011B000DFCFC4F0010EDBCFC5F0020EDBCFC6F0EF
:1011C000030EDBCFC7F0070EE76EFD0EDBCFE9FFA6
:1011D000FE0EDBCFEAFFE750E926000EEA22EF50D1
:1011E000800B02E00001C78FA2EC12F0020EE76E46
:1011F000FD0EDBCFE9FFFE0EDBCFEAFFE750E9266D
:10120000000EEA22EF50FF0810E0020EE76EFD0E1E
:10121000DBCFE9FFFE0EDBCFEAFFE750E926000E49
:10122000EA22EF50E66E07D8E552D9CFE1FFE5524A
:10123000E7CFD9FF1200D9CFE6FFE1CFD9FF080EE3
:10124000E126E8680001C41908E1E868C51905E16C
:10125000E868C61902E1E868C71901E188D0CD0540
:1012600001E185D0080EE66EE66AE66AD9CFE6FFB0
:10127000DACFE6FF4CEC30F0F56E050EE15EF5508E
:10128000FE0EDB50006E016AD890015004E6800E1D
:10129000005C000E015811E3D9CFE6FFDACFE6FF7C
:1012A000FE0EDBCFE6FF2CEC24F0E552E552E552D2
:1012B000000902E0010E5DD042D0FE0EDB50010AB3
:1012C00021E0010A02E0010E54D0050EE66EE66A46
:1012D000D1EC1EF0F3CF00F0F4CF01F0026A00C0B1
:1012E000E6FF01C0E6FF02C0E6FFD950020FE66E3E
:1012F000000EDA20E66E29EC30F0F56E070EE15EA6
:10130000F5501DD0050EE66EE66ADBEC1EF0F3CF5D
:1013100000F0F4CF01F0026A00C0E6FF01C0E6FF72
:1013200002C0E6FFD950020FE66E000EDA20E66E2C
:1013300029EC30F0F56E070EE15EF55000D0DF6A63
:10134000FE0EDB50E76E010EE7CFDBFFE66E080E08
:10135000E66ED9CFE6FFDACFE6FF010EE66EBAEC15
:1013600015F0F56E050EE15EF55003D002D0000ECB
:1013700000D0D9CFE1FFE552E7CFD9FF1200D9CF96
:10138000E6FFE1CFD9FF0D0EE126020EE76EFD0E5E
:10139000DBCFE9FFFE0EDBCFEAFFE750E926000EC8
:1013A000EA22EFCF00F0016A026A036A030EE76ED9
:1013B000FD0EDBCFE9FFFE0EDBCFEAFFE750E926AB
:1013C000000EEA22EFCF04F0056A066A076A080EEB
:1013D0001F0B07E0D8900436053606360736E806B8
:1013E000F9E1045000260550012206500222075060
:1013F0000322040EE76EFD0EDBCFE9FFFE0EDBCF0E
:10140000EAFFE750E926000EEA22EFCF08F0096A6A
:101410000A6A0B6A100E1F0B07E0D89008360936CF
:101420000A360B36E806F9E1085000260950012279
:101430000A5002220B500322050EE76EFD0EDBCF91
:10144000E9FFFE0EDBCFEAFFE750E926000EEA22B5
:10145000EF501F0B0C6E0D6A0E6A0F6A180E1F0BF1
:1014600007E0D8900C360D360E360F36E806F9E157
:101470000C5000260D5001220E5002220F50032264
:1014800000C0DFFF010E01C0DBFF020E02C0DBFF68
:10149000030E03C0DBFF050EE76EFD0EDBCFE9FF99
:1014A000FE0EDBCFEAFFE750E926000EEA22EF50FE
:1014B000800BE76E040EE7CFDBFF060EE76EFD0E36
:1014C000DBCFE9FFFE0EDBCFEAFFE750E926000E97
:1014D000EA22050EEFCFDBFF070EE76EFD0EDBCF36
:1014E000E9FFFE0EDBCFEAFFE750E926000EEA2215
:1014F000EF50010BE76E060EE7CFDBFF070EE76E3E
:10150000FD0EDBCFE9FFFE0EDBCFEAFFE750E92659
:10151000000EEA22EF407F0BE76E070EE7CFDBFFFE
:10152000DB50020A01E117D2010A01E145D1020AAA
:1015300001E179D0010A01E0A7D2010EF36E0B0E92
:10154000F3CFDBFF040EDB5002E00B0EDB880A0E4C
:10155000DB6A0C0EF36E0A0EDBCFF4FFF350F45C83
:1015600061E20A0EDB50080DF3CFE9FFF4CFEAFF8A
:10157000600EE926000EEA22EECF00F0EECF01F079
:10158000EECF02F0EFCF03F0D9CFE9FFDACFEAFFD9
:101590000050EE1809E10150EE1806E10250EE1875
:1015A00003E10350EE1800E13AE10A0EDB50080DAA
:1015B000F3CFE9FFF4CFEAFF600EE926000EEA223E
:1015C000070EE926000EEA22EF50110B046E0B0EF7
:1015D000DB50045C24E1060EDB5011E00A0EDB5008
:1015E000080DF3CFE9FFF4CFEAFF600EE926000E05
:1015F000EA22070EE926000EEA22EF8210D00A0E38
:10160000DB50080DF3CFE9FFF4CFEAFF600EE926C7
:10161000000EEA22070EE926000EEA22EF920A0ED9
:10162000DB2A97D731D2050EDBCFE6FF2FEC06F091
:10163000E552080EF3CFDBFF090EF4CFDBFF080EF7
:10164000DBCF00F0090EDBCF01F00001800E0114AA
:1016500016E0E66AE668E668E668E668E66AE66A6C
:10166000050EDBCFE6FF6FEC06F0F56E080EE15ECF
:10167000F550080EF3CFDBFF090EF4CFDBFF080EA9
:10168000DBCF00F0090EDBCF01F00001800E01146A
:1016900001E0FAD1080EDBCF00F0090EDBCF01F03C
:1016A000800E011401E087D0080EDBCFE9FF090EA0
:1016B000DBCFEAFF030ED890E936EA36E806FBE115
:1016C000600EE926000EEA22DFCFEEFF010EDBCF2F
:1016D000EEFF020EDBCFEEFF030EDBCFEEFF040EBC
:1016E000DB5016E0080EDBCFE9FF090EDBCFEAFF87
:1016F000030ED890E936EA36E806FBE1600EE926EB
:10170000000EEA22070EE926000EEA22EF8815D025
:10171000080EDBCFE9FF090EDBCFEAFF030ED890FE
:10172000E936EA36E806FBE1600EE926000EEA2219
:10173000070EE926000EEA22EF98060EDB5016E0AF
:10174000080EDBCFE9FF090EDBCFEAFF030ED890CE
:10175000E936EA36E806FBE1600EE926000EEA22E9
:10176000070EE926000EEA22EF8215D0080EDBCF25
:10177000E9FF090EDBCFEAFF030ED890E936EA361F
:10178000E806FBE1600EE926000EEA22070EE926D4
:10179000000EEA22EF92080EDBCFE6FF090EDBCF48
:1017A000E6FF84EC07F0E552E552080EF3CFDBFFCD
:1017B000090EF4CFDBFF68D1050EDBCFE6FF2FEC7F
:1017C00006F0E552080EF3CFDBFF090EF4CFDBFF86
:1017D000080EDBCF00F0090EDBCF01F00001800E18
:1017E000011416E0E66AE668E668E668E668E66A16
:1017F000E66A050EDBCFE6FF6FEC06F0F56E080E2D
:10180000E15EF550080EF3CFDBFF090EF4CFDBFFEE
:10181000080EDBCF00F0090EDBCF01F00001800ED7
:10182000011401E031D10C0EDB6A010EF36E0B0ED8
:10183000F3CFDBFF040EDB5002E00B0EDB880A0E59
:10184000DB6A0C0EF36E0A0EDBCFF4FFF350F45C90
:1018500001E380D00A0EDB50080DF3CFE9FFF4CF8F
:10186000EAFF600EE926000EEA22070EE926000EC6
:10187000EA22EF50110B006E0B0EDB50005C67E1AB
:101880000A0EDB50080DF3CFE9FFF4CFEAFF600E3C
:10189000E926000EEA22EECF01F0EECF02F0EECF05
:1018A00003F0EFCF04F0D9CFE9FFDACFEAFF015020
:1018B000EE1809E10250EE1806E10350EE1803E1BC
:1018C0000450EE1800E143E10C0EDB5038E10A0E43
:1018D000DB50006E016A080EDB50001803E1090EB0
:1018E000DB5001182BE0080EDBCF00F0090EDBCF38
:1018F00001F00001800E01140AE1080EDBCFE6FFC3
:10190000090EDBCFE6FF97EC07F0E552E5520A0E31
:10191000DB50080DF3CFE9FFF4CFEAFF600EE926B4
:10192000000EEA22060EE926000EEA22050EDBCFA3
:10193000EFFF010EF36E0C0EF3CFDBFF08D00A0EA3
:10194000DBCFE6FFE66A97EC07F0E552E5520A0EB8
:10195000DB2A77D799D0060EDB5001E094D0010E38
:10196000F36E0B0EF3CFDBFF040EDB5002E00B0E29
:10197000DB880A0EDB6A0C0EF36E0A0EDBCFF4FF77
:10198000F350F45C01E37FD00A0EDB50080DF3CF77
:10199000E9FFF4CFEAFF600EE926000EEA22070E07
:1019A000E926000EEA22EF50110B006E0B0EDB5001
:1019B000005C66E10A0EDB50080DF3CFE9FFF4CFBF
:1019C000EAFF600EE926000EEA22EECF01F0EECF2C
:1019D00002F0EECF03F0EFCF04F0D9CFE9FFDACF7A
:1019E000EAFF0150EE1809E10250EE1806E103503B
:1019F000EE1803E10450EE1800E142E10A0EDB505C
:101A0000080DF3CFE9FFF4CFEAFF600EE926000EE0
:101A1000EA22070EE926000EEA22EF50400B09E108
:101A20000A0EDBCFE6FFE66A97EC07F0E552E552D7
:101A300027D00A0EDB50080DF3CFE9FFF4CFEAFF01
:101A4000600EE926000EEA22070EE926000EEA22C1
:101A5000EF920A0EDB50080DF3CFE9FFF4CFEAFF57
:101A6000600EE926000EEA22EE68EE68EE68EE6887
:101A70000A0EDBCFE6FFE66A84EC07F0E552E5529A
:101A80000A0EDB2A78D700D0D9CFE1FFE552E7CFA5
:101A9000D9FF1200D9CFE6FFE1CFD9FF020EE12630
:101AA000DF6E080EDF5C72E2DF50E76EFD0EDBCF0B
:101AB000E9FFFE0EDBCFEAFFE750E926000EEA223F
:101AC000EF5001E163D0010EDB6A040EF36E010EEC
:101AD000DBCFF4FFF350F45C1CE2010EDB50EA6A4A
:101AE000C00FE96E000EEA22EFCF00F0DF50E76E84
:101AF000FD0EDBCFE9FFFE0EDBCFEAFFE750E92664
:101B0000000EEA22EF50005C01E103D0010EDB2A57
:101B1000DCD7010EDB50040837E1010EDB6A040E4E
:101B2000F36E010EDBCFF4FFF350F45C0DE2010E17
:101B3000DB50EA6AC00FE96E000EEA22EF5001E1C5
:101B400003D0010EDB2AEBD7040EF36E010EDBCFC0
:101B5000F4FFF350F45C18E2DF50E76EFD0EDBCFCC
:101B6000E9FFFE0EDBCFEAFFE750E926000EEA228E
:101B7000EF50E66E010EDB50EA6AC00FE96E000E10
:101B8000EA22E552E750EF6EDF2A8BD7D9CFE1FF8B
:101B9000E552E7CFD9FF1200D9CFE6FFE1CFD9FF59
:101BA000040EE126020EDE6EDD6ADECF00F0DDCF30
:101BB00001F0D890015004E6080E005C000E0158B8
:101BC00001E3E9D0FD0EDBCF00F0FE0EDBCF01F02C
:101BD000DE500024E96EDD500120EA6EEF5001E195
:101BE000DAD0020EDB6A030EDB6A020EDBCF00F0F6
:101BF000030EDBCF01F0D890015004E6040E005C28
:101C0000000E01582EE2020EDBCFE9FF030EDBCF00
:101C1000EAFFC00EE926000EEA22EF501BE0020E9A
:101C2000DBCFE9FF030EDBCFEAFFC00EE926000E93
:101C3000EA22EFCF00F0FD0EDBCF01F0FE0EDBCF8E
:101C400002F0DE500124E96EDD500220EA6EEF5012
:101C5000005C01E106D0020EDB2A030E01E3DB2A61
:101C6000C4D7020EDBCF00F0030EDBCF01F0D8901B
:101C7000015004E6040E005C000E015801E386D01A
:101C8000020EDBCFE9FF030EDBCFEAFFC00EE92631
:101C9000000EEA22EF5001E179D0020EDBCFE9FF1E
:101CA000030EDBCFEAFFC00EE926000EEA22EF6A40
:101CB000010EE76E020EDBCF00F0030EDBCF01F06A
:101CC000E7500026000E012200C0DEFF01C0DDFF4C
:101CD000DECF00F0DDCF01F0D890015004E6040E15
:101CE000005C000E015810E2DECFE9FFDDCFEAFF15
:101CF000C00EE926000EEA22EF5001E105D0DF2AEE
:101D0000010E01E3DB2AE4D7DECF00F0DDCF01F0E6
:101D1000D890015004E6040E005C000E015836E233
:101D2000010EE76E020EDBCF02F0030EDBCF03F0F5
:101D3000E7500226000E03220250DF1803E1035091
:101D4000DE52DD1823E0DECFE9FFDDCFEAFFE90652
:101D5000000EEA5AC00EE926000EEA22EF50E66EA7
:101D6000020EDBCFE9FF030EDBCFEAFFC00EE92650
:101D7000000EEA22E552E750EF6EDECFE9FFDDCF3D
:101D8000EAFFC00EE926000EEA22EF6ADF2A010E02
:101D900001E3DB2A0AD7D9CFE1FFE552E7CFD9FF2C
:101DA0001200D9CFE6FFE1CFD9FF020EE76EFD0E9C
:101DB000DBCFE9FFFE0EDBCFEAFFE750E926000E9E
:101DC000EA22EF5006082BE1040EE76EFD0EDBCF92
:101DD000E9FFFE0EDBCFEAFFE750E926000EEA221C
:101DE000EFCFC9F0050EE76EFD0EDBCFE9FFFE0E6B
:101DF000DBCFEAFFE750E926000EEA22EFCFCAF078
:101E0000060EE76EFD0EDBCFE9FFFE0EDBCFEAFF2D
:101E1000E750E926000EEA22EFCFCBF02CDBE552AB
:101E2000E7CFD9FF1200D9CFE6FFE1CFD9FF030EEC
:101E3000E76EFD0EDBCFE9FFFE0EDBCFEAFFE750DA
:101E4000E926000EEA22EFCFC8F07CDB020EE76E37
:101E5000FD0EDBCFE9FFFE0EDBCFEAFFE750E92600
:101E6000000EEA22EF50FF0811E0020EE76EFD0EB1
:101E7000DBCFE9FFFE0EDBCFEAFFE750E926000EDD
:101E8000EA22EF50E66E1BEC09F0E552E552E7CF8F
:101E9000D9FF1200D9CFE6FFE1CFD9FF0A0EE12624
:101EA000020EE76EFD0EDBCFE9FFFE0EDBCFEAFF91
:101EB000E750E926000EEA22EFCFDFFF040EE76EBF
:101EC000FD0EDBCFE9FFFE0EDBCFEAFFE750E92690
:101ED000000EEA22EF50010BE76E010EE7CFDBFFA9
:101EE000040EE76EFD0EDBCFE9FFFE0EDBCFEAFF4F
:101EF000E750E926000EEA22EF50100BE76E020EC3
:101F0000E7CFDBFF040EE76EFD0EDBCFE9FFFE0E31
:101F1000DBCFEAFFE750E926000EEA22EF50200B64
:101F2000E76E030EE7CFDBFF040EE76EFD0EDBCF9F
:101F3000E9FFFE0EDBCFEAFFE750E926000EEA22BA
:101F4000EF50400BE76E040EE7CFDBFF050EE76EA8
:101F5000FD0EDBCFE9FFFE0EDBCFEAFFE750E926FF
:101F6000000EEA22EFCF02F002C003F0026A060E72
:101F7000E76EFD0EDBCFE9FFFE0EDBCFEAFFE75099
:101F8000E926000EEA22EF5000010224006E000E46
:101F90000320016E050E00C0DBFF060E01C0DBFF53
:101FA000020EDF5C01E2E7D1DFCFE6FF2FEC06F0A7
:101FB000E552070EF3CFDBFF080EF4CFDBFF030E75
:101FC000DB500EE0020EDB500BE1070EDBCF00F022
:101FD000080EDBCF01F00001800E011401E0CBD12F
:101FE000070EDBCF00F0080EDBCF01F00001800E02
:101FF000011415E0E66AE668E668E668E668E66AFF
:10200000E66ADFCFE6FF6FEC06F0F56E080EE15EE4
:10201000F550070EF3CFDBFF080EF4CFDBFF070E02
:10202000DBCF00F0080EDBCF01F00001800E0114C1
:1020300001E0A1D1030EE76EFD0EDBCFE9FFFE0E3E
:10204000DBCFEAFFE750E926000EEA22EF5001E17C
:1020500091D0030EE76EFD0EDBCFE9FFFE0EDBCF66
:10206000EAFFE750E926000EEA22EF500F0BE76E79
:10207000090EE7CFDBFFDB5008082DE3070EDBCFAF
:10208000E9FF080EDBCFEAFF030ED890E936EA3607
:10209000E806FBE1600EE926000EEA22050EE926BD
:1020A000000EEA22090EDBCFEFFF070EDBCFE9FFC0
:1020B000080EDBCFEAFF030ED890E936EA36E806D1
:1020C000FBE1600EE926000EEA22070EE926000E6B
:1020D000EA22EF8A15D0070EDBCFE9FF080EDBCF2F
:1020E000EAFF030ED890E936EA36E806FBE1600E17
:1020F000E926000EEA22070EE926000EEA22EF9AF0
:10210000030EE76EFD0EDBCFE9FFFE0EDBCFEAFF2D
:10211000E750E926000EEA22EF50400B16E0070ECA
:10212000DBCFE9FF080EDBCFEAFF030ED890E936DC
:10213000EA36E806FBE1600EE926000EEA22070E09
:10214000E926000EEA22EF8615D0070EDBCFE9FF65
:10215000080EDBCFEAFF030ED890E936EA36E80630
:10216000FBE1600EE926000EEA22070EE926000ECA
:10217000EA22EF96040EE76EFD0EDBCFE9FFFE0EBE
:10218000DBCFEAFFE750E926000EEA22EF5001E13B
:10219000A4D0020EDB502DE0070EDBCFE9FF080EC6
:1021A000DBCFEAFF030ED890E936EA36E806FBE11A
:1021B000600EE926000EEA22040EE926000EEA224D
:1021C000050EDBCFEFFF070EDBCFE9FF080EDBCFFD
:1021D000EAFF030ED890E936EA36E806FBE1600E26
:1021E000E926000EEA22070EE926000EEA22EF8C0D
:1021F00018D0030EDB5015E0070EDBCFE9FF080E09
:10220000DBCFEAFF030ED890E936EA36E806FBE1B9
:10221000600EE926000EEA22070EE926000EEA22E9
:10222000EF9C040EDB5016E0070EDBCFE9FF080E33
:10223000DBCFEAFF030ED890E936EA36E806FBE189
:10224000600EE926000EEA22070EE926000EEA22B9
:10225000EF8215D0070EDBCFE9FF080EDBCFEAFFD8
:10226000030ED890E936EA36E806FBE1600EE9266F
:10227000000EEA22070EE926000EEA22EF92010E76
:10228000DB5016E0070EDBCFE9FF080EDBCFEAFFDD
:10229000030ED890E936EA36E806FBE1600EE9263F
:1022A000000EEA22070EE926000EEA22EF8415D07E
:1022B000070EDBCFE9FF080EDBCFEAFF030ED89055
:1022C000E936EA36E806FBE1600EE926000EEA226E
:1022D000070EE926000EEA22EF94070EDBCFE9FF96
:1022E000080EDBCFEAFF030ED890E936EA36E8069F
:1022F000FBE1600EE926000EEA22E868EE1808E12C
:10230000E868EE1805E1E868EE1802E1E868EE1802
:1023100022E1070EDBCFE9FF080EDBCFEAFF030E59
:10232000D890E936EA36E806FBE1600EE926000EB1
:10233000EA22070EE926000EEA22EF50400B0BE1DD
:10234000070EDBCFE6FF080EDBCFE6FF97EC07F0CA
:10235000E552E55210D0070EDBCFE6FF080EDBCFCB
:10236000E6FF84EC07F0E552E552070EF3CFDBFF02
:10237000080EF4CFDBFFD9CFE1FFE552E7CFD9FF5D
:102380001200D9CFE6FFE1CFD9FF080EE126020EF9
:10239000E76EFD0EDBCFE9FFFE0EDBCFEAFFE75075
:1023A000E926000EEA22EF50060A46E0030A24E07E
:1023B000010A1BE0070A17E0010A13E0030A0AE01A
:1023C000010A01E052D0010EE66EE66A82D8E552BB
:1023D000E5524BD0E66A010EE66E7BD8E552E55237
:1023E00044D062D942D001DA40D0010EE66EE66AEE
:1023F00060D9E552E55239D0040EE76EFD0EDBCF11
:10240000E9FFFE0EDBCFEAFFE750E926000EEA22E5
:10241000EF50E66E030EE76EFD0EDBCFE9FFFE0E1A
:10242000DBCFEAFFE750E926000EEA22EF50E66E26
:10243000E1D9E552E55219D0D9CFE6FFDACFE6FF70
:10244000ACEC1EF0E552E55200090EE1070EDBCFC1
:10245000E6FF060EDBCFE6FF050EDBCFE6FFB2ECB4
:1024600017F0E552E552E55200D0D9CFE1FFE55231
:10247000E7CFD9FF1200D9CFE6FFE1CFD9FF080E91
:10248000E126C40EE66E000EE66EACEC1EF0E552E0
:10249000E552000904E0010EF36EF46A14D0050E53
:1024A000C9C0DBFF060ECAC0DBFF070ECBC0DBFFD7
:1024B000D9CFE6FFDACFE6FFC9EC1EF0E552E552D0
:1024C000F36AF46A00D0D9CFE1FFE552E7CFD9FF34
:1024D0001200D9CFE6FFE1CFD9FF080EE126C40EE6
:1024E000E66E000EE66EACEC1EF0E552E552000919
:1024F00004E0010EF36EF46A1FD0FE0EDB5003E021
:10250000040EC8C0DBFFFD0EDB500BE0C4C0DFFFD4
:10251000010EC5C0DBFF020EC6C0DBFF030EC7C045
:10252000DBFFD9CFE6FFDACFE6FFC9EC1EF0E552BC
:10253000E552F36AF46A00D0D9CFE1FFE552E7CF64
:10254000D9FF1200D9CFE6FFE1CFD9FF020EE12675
:10255000010EE66EE66EF7EC04F0E552E552F3CFBD
:10256000DEFFF4CFDDFFDECF00F0DDCF01F00001B4
:10257000800E011401E092D0E8680001C41908E15E
:10258000E868C51905E1E868C61902E1E868C719F5
:1025900067E0C4C000F0C5C001F0C6C002F0C7C00B
:1025A00003F01F0E0316C8C004F0056A066A076A26
:1025B0000450002605500122065002220750032233
:1025C000DECFE9FFDDCFEAFF030ED890E936EA3629
:1025D000E806FBE1600EE926000EEA2200C0EEFFED
:1025E00001C0EEFF02C0EEFF03C0EEFFC4C000F06A
:1025F000C5C001F0C6C002F0C7C003F0006A016A9E
:10260000026A800E0316005001100210031014E03D
:10261000DECFE9FFDDCFEAFF030ED890E936EA36D8
:10262000E806FBE1600EE926000EEA22070EE92625
:10263000000EEA22EF8813D0DECFE9FFDDCFEAFFFC
:10264000030ED890E936EA36E806FBE1600EE9268B
:10265000000EEA22070EE926000EEA22EF9812D0B9
:10266000DECFE9FFDDCFEAFF030ED890E936EA3688
:10267000E806FBE1600EE926000EEA22EE68EE684D
:10268000EE68EE68DECFE6FFDDCFE6FF84EC07F014
:10269000E552E552F3CFDEFFF4CFDDFFD9CFE1FF06
:1026A000E552E7CFD9FF1200010EF36EF46A00D0B5
:1026B0001200D9CFE6FFE1CFD9FF020EE126DE6A94
:1026C000DD6ADECF00F0DDCF01F0D890015004E6E6
:1026D0000C0E005C000E015822E2DECFE9FFDDCFD8
:1026E000EAFF030ED890E936EA36E806FBE1600E11
:1026F000E926000EEA22070EE926000EEA22EF5034
:10270000010B08E0DECFE6FFDDCFE6FF97EC07F038
:10271000E552E552DF2A010E01E3DB2AD2D7D95078
:10272000FD0FE96EFF0EDA20EA6EEE50ED1057E075
:10273000E66AE66AE66A010EE66E080EE66EE66A8C
:10274000E66AE66AE66AE66AE66A78EC01F0F56E41
:102750000B0EE15EF550C4C000F0C5C001F0C6C06C
:1027600002F0C7C003F0006A016A026A800E031615
:10277000005001100210031002E1000E01D0010E02
:10278000E66E010EE66EE66EE66E080EE66EC4C0FC
:1027900004F0C5C005F0C6C006F0C7C007F01F0EA4
:1027A0000716C8C008F0096A0A6A0B6A08500426AE
:1027B000095005220A5006220B50072204C0E6FFEA
:1027C00005C0E6FF06C0E6FF07C0E6FF010EE66EA5
:1027D000E66E78EC01F0F56E0B0EE15EF550D9CFA8
:1027E000E1FFE552E7CFD9FF1200010EF36EF46A64
:1027F00000D01200D9CFE6FFE1CFD9FF090EE126C4
:10280000FD0EDB50006E016AA00E001801E10150C0
:102810000DE0FD0EDB50026E036AA10E021801E10D
:10282000035004E0010EF36EF46A9ED1DF6A0C0ED1
:10283000DF5C19E2DF50080DF3CFE9FFF4CFEAFFC8
:10284000600EE926000EEA22070EE926000EEA22B3
:10285000EF50010B06E0FE0EDB5001E104D0FE0E4E
:10286000DB06DF2AE4D7010EDB6AFD0EDB50E76EE4
:10287000020EE7CFDBFF0C0EDF5C17E1080EDB6812
:10288000010EE66E080EE66ED950010FE66E000EE0
:10289000DA20E66E010EE66E6DD9F56E050EE15E8C
:1028A000F550010EF36EF46A5FD1FD0EDB50006E41
:1028B000016AA00E001801E1015001E0B2D0DF5022
:1028C000080DF3CFE9FFF4CFEAFF600EE926000E12
:1028D000EA22EECF00F0EECF01F0EECF02F0EFCF24
:1028E00003F00050E76E030EE7CFDBFFDF50080D6B
:1028F000F3CFE9FFF4CFEAFF600EE926000EEA22EB
:10290000EECF00F0EECF01F0EECF02F0EFCF03F00C
:10291000080ED8900332023201320032E806F9E1A3
:102920000050E76E040EE7CFDBFFDF50080DF3CF5A
:10293000E9FFF4CFEAFF600EE926000EEA22EECFAF
:1029400000F0EECF01F0EECF02F0EFCF03F0100E6B
:10295000D8900332023201320032E806F9E1005029
:10296000E76E050EE7CFDBFFDF50080DF3CFE9FF81
:10297000F4CFEAFF600EE926000EEA22EECF00F067
:10298000EECF01F0EECF02F0EFCF03F0180ED890AB
:102990000332023201320032E806F9E10050E76EFC
:1029A000060EE7CFDBFFDF50080DF3CFE9FFF4CFD2
:1029B000EAFF600EE926000EEA22070EE926000E65
:1029C000EA22EF50100B02E0060EDB8EDF50080DFE
:1029D000F3CFE9FFF4CFEAFF600EE926000EEA220A
:1029E000060EE926000EEA22070EEFCFDBFFDF50CE
:1029F000080DF3CFE9FFF4CFEAFF600EE926000EE1
:102A0000EA22070EE926000EEA22EF50020B06E04A
:102A1000010EF36E080EF3CFDBFF02D0080EDB6A67
:102A20008BD0DF50080DF3CFE9FFF4CFEAFF600E43
:102A3000E926000EEA22060EE926000EEA22030E1F
:102A4000EFCFDBFFDF50080DF3CFE9FFF4CFEAFF54
:102A5000600EE926000EEA22070EE926000EEA22A1
:102A6000EF50200B10E0DF50080DF3CFE9FFF4CF5B
:102A7000EAFF600EE926000EEA22050EE926000EA6
:102A8000EA22EF5001D00F0E800FE76E040EE7CF61
:102A9000DBFFDF50080DF3CFE9FFF4CFEAFF600E54
:102AA000E926000EEA22070EE926000EEA22EF5080
:102AB000080B02E0040EDB8C800EF36E050EF3CFE4
:102AC000DBFFDF50080DF3CFE9FFF4CFEAFF600E24
:102AD000E926000EEA22070EE926000EEA22EF5050
:102AE000020B02E0050EDB8CDF50080DF3CFE9FF8F
:102AF000F4CFEAFF600EE926000EEA22070EE9266F
:102B0000000EEA22EF50040B02E0050EDB80060EF9
:102B1000DB6ADF50080DF3CFE9FFF4CFEAFF600E68
:102B2000E926000EEA22040EE926000EEA22070E2C
:102B3000EFCFDBFF080EDB6A010EE66E080EE66ED5
:102B4000D950010FE66E000EDA20E66E010EE66E39
:102B500011D8F56E050EE15EF550006E016A00C0F9
:102B6000F3FF01C0F4FF00D0D9CFE1FFE552E7CF7A
:102B7000D9FF1200D9CFE6FFE1CFD9FF030EE1263E
:102B80000001CC0508E0FE0EDB0405E0FA0EDB5088
:102B900002E1010EBCD0CD0502E1010EB8D0020E5B
:102BA000CD5D05E1FE0EDB0402E0010EB0D037EC96
:102BB00024F0010EE66EFE0EDBCFE6FFF7EC04F02C
:102BC000E552E552F3CFDEFFF4CFDDFFDECF00F0BC
:102BD000DDCF01F00001800E011430E1DECFE9FF0E
:102BE000DDCFEAFF030ED890E936EA36E806FBE1CE
:102BF000600EE926000EEA22070EE926000EEA2200
:102C0000EF50030B03081AE1DECFE9FFDDCFEAFF47
:102C1000030ED890E936EA36E806FBE1600EE926B5
:102C2000000EEA22E868EE1808E1E868EE1805E10F
:102C3000E868EE1802E1E868EE1804E138EC24F0E8
:102C4000010E65D0DECFE9FFDDCFEAFF030ED8909D
:102C5000E936EA36E806FBE1600EE926000EEA22D4
:102C6000070EE926000EEA22EF50200B15E0DECF1A
:102C7000E9FFDDCFEAFF030ED890E936EA36E80631
:102C8000FBE1600EE926000EEA22050EE926000EA1
:102C9000EA22FB0EEFCFDBFFFB0EDBCFE6FFFC0EE5
:102CA000DBCFE6FFFD0EDBCFE6FFDECFE9FFDDCFBA
:102CB000EAFF030ED890E936EA36E806FBE1600E3B
:102CC000E926000EEA22EECFE6FFEECFE6FFEECFDA
:102CD000E6FFEFCFE6FF66EC18F0F56E070EE15E5B
:102CE000F550E76E020EE7CFDBFF38EC24F0020E62
:102CF000DB5003E1000E0BD00AD0CC0EE66E600E66
:102D0000E66EA5EC2CF0E552E552010E00D0D9CFCD
:0A2D1000E1FFE552E7CFD9FF120002
:062D1A00D9CFE6FFE1CF76
:102D2000D9FF100EE126B00E9C6EDF6A3EEC27F054
:102D300009EC2FF0E6EC1EF0010EE66E57EC00F009
:102D4000E5520101090511E18B0EE66E610EE66E9A
:102D5000A5EC2CF0E552E552690EE66E610EE66ECA
:102D6000A5EC2CF0E552E55220D0020E0101095DE0
:102D700009E1550EE66E610EE66EA5EC2CF0E5520B
:102D8000E55213D0420EE66E610EE66EA5EC2CF015
:102D9000E552E55201010951E66EE66AAAEC2DF012
:102DA000E552E552C7EC2CF0FFD70101090501E11E
:102DB00002D0829A949A010EDF6EDF501CE0DFCFC2
:102DC000E6FF50EC27F0E5520A0EE66EE66A7AEC72
:102DD0002FF0E552E552F3CF00F0F4CF01F000C040
:102DE000E6FF01C0E6FFA0EC2FF0E552E552DF5010
:102DF000E824DF6EE2D7800EDF6EDF501CE0DFCF0D
:102E0000E6FF50EC27F0E5520A0EE66EE66A7AEC31
:102E10002FF0E552E552F3CF00F0F4CF01F000C0FF
:102E2000E6FF01C0E6FFA0EC2FF0E552E552DF40DF
:102E30007F0BDF6EE2D7E66A50EC27F0E552010126
:102E4000090501E0828A0001FE0EDE6F040087ECB6
:102E50002CF0000901E050D0D950070FE66E000EAB
:102E6000DA20E66ED950080FE66E000EDA20E66E24
:102E7000D950030FE66E000EDA20E66EA1D8F56E8B
:102E8000060EE15EF550E76E010EE7CFDBFF010EA7
:102E9000DB501CE1070EDBCFE6FFD950080FE66ED2
:102EA000000EDA20E66ED950030FE96EDACFEAFFA2
:102EB000EECFE6FFEECFE6FFEECFE6FFEFCFE6FF89
:102EC00074EC02F0F56E070EE15EF55001010905A4
:102ED00006E1DFD9E76E020EE7CFDBFF02D0020E7C
:102EE000DB6A15EC1FF0010EDB5005E0020EDB5033
:102EF00002E1D3EC2FF0AAD7D9CFE1FFE552E7CF1B
:102F0000D9FF1200D9CFE6FFE1CFD9FFE652010188
:102F1000165113E1FC0EDBCFE6FFFD0EDBCFE6FF23
:102F2000FE0EDBCFE6FF39EC24F0E552E552E55228
:102F3000DF6E0101010E166F0ED0FC0EDBCFE6FF37
:102F4000FD0EDBCFE6FFFE0EDBCFE6FF0BD8E55232
:102F5000E552E552DF6EDF5000D0E552E552E7CF93
:102F6000D9FF1200D9CFE6FFE1CFD9FF01011651F9
:102F700010E0FC0EDBCFE6FFFD0EDBCFE6FFFE0E22
:102F8000DBCFE6FF77EC24F0E552E552E55203D0C3
:102F900002D0000E00D0E552E7CFD9FF1200D9CF02
:102FA000E6FFE1CFD9FF0101165106E0FE0EDBCFAF
:102FB000E6FF97EC24F0E552E552E7CFD9FF120087
:102FC000D9CFE6FFE1CFD9FFE6520101165175E0F6
:102FD000F90EDBCFE6FFFA0EDBCFE6FFFB0EDBCF11
:102FE000E6FFFC0EDBCFE6FFFD0EDBCFE6FFFE0EBD
:102FF000DBCFE6FFEFEC24F0F56E060EE15EF55058
:10300000DF6EDF5059E10101155125E0F90EDBCFEC
:10301000E9FFFA0EDBCFEAFFEF50E66EFB0EDBCFE7
:10302000E6FFFC0EDBCFE6FFFD0EDBCFE9FFFE0E79
:10303000DBCFEAFFEECFE6FFEECFE6FFEECFE6FF17
:10304000EFCFE6FFF7DAF56E070EE15EF55000010F
:10305000FE0EDE6F31D0FD0EDBCFE9FFFE0EDBCFC3
:10306000EAFFEECFD1F0EECFD2F0EECFD3F0EFCF3C
:10307000D4F0F90EDBCFE9FFFA0EDBCFEAFFEFCF9A
:10308000D5F0F90EDBCFE9FFFA0EDBCFEAFFEF5008
:10309000E66EE66AFB0EDBCFE6FFFC0EDBCFE6FF5B
:1030A000D60EE66E000EE66EFEEC2FF0F56E060E06
:1030B000E15EF5500001DE6B02D0FE0EDF6EDF50E8
:1030C00000D0E552E552E7CFD9FF1200D9CFE6FF95
:1030D000E1CFD9FFE652010116511FE0F80EDBCF18
:1030E000E6FFF90EDBCFE6FFFA0EDBCFE6FFD950A5
:1030F000FB0FE96EFF0EDA20EA6EEECFE6FFEECFB1
:10310000E6FFEECFE6FFEFCFE6FFE8EC25F0F56E49
:10311000070EE15EF550DF6E01D0DF6A0101155147
:1031200020E0F80EDBCFE6FFF90EDBCFE6FFFA0E6C
:10313000DBCFE6FFD950FB0FE96EFF0EDA20EA6E17
:10314000EECFE6FFEECFE6FFEECFE6FFEFCFE6FFF6
:1031500071DAF56E070EE15EF5500001FE0EDE6FCE
:1031600024D0FB0EDBCFD1F0FC0EDBCFD2F0FD0E76
:10317000DBCFD3F0FE0EDBCFD4F0F80EDBCFD5F0F3
:10318000DBCFE6FFE66AF90EDBCFE6FFFA0EDBCF18
:10319000E6FFD60EE66E000EE66EFEEC2FF0F56E44
:1031A000060EE15EF5500001DE6BDF5000D0E55207
:1031B000E552E7CFD9FF12000101165104E0B8EC47
:1031C00024F00101166B1200D9CFE6FFE1CFD9FF41
:1031D000300E006EFE0EDBCFE7FF0050E75EFE0E06
:1031E000E7CFDBFFDB5009080AE2070E006EFE0E98
:1031F000DBCFE7FF0050E75EFE0EE7CFDBFFFE0E02
:10320000DB500F080AE2200E006EFE0EDBCFE7FF58
:103210000050E75EFE0EE7CFDBFFFE0EDB5000D076
:10322000E552E7CFD9FF1200D9CFE6FFE1CFD9FFB2
:10323000FE0EDBCFE6FFC8DFE552E76EFE0EE7CFFE
:10324000DBFFFD0EDBCFE6FFBFDFE552E76EFD0ED5
:10325000E7CFDBFFFE0EDB500F0814E3FD0EDB5063
:103260000F0810E3FD0EDBCFE6FFFE0EDB38F00BA0
:10327000E552E724006E016A00C0F3FF01C0F4FFCD
:1032800004D003D0F368F46800D0E552E7CFD9FF4B
:103290001200D9CFE6FFE1CFD9FF030EE126020EDF
:1032A000DB6AE6EC2EF0F3CFDEFFF4CFDDFFDECFFE
:1032B00000F0DDCF01F00001800E011401E0FFD02D
:1032C000010EF36E020EF3CFDBFF01011851020A6B
:1032D0006CE0010A6AE0020A2AE0010A01E000D07B
:1032E000D9CFE9FFDACFEAFF020EEE1801E1ED5087
:1032F00009E0D9CFE9FFDACFEAFF4D0EEE1801E180
:10330000ED5014E10001F16B0101010E186FD9CFEE
:10331000E9FFDACFEAFF4D0EEE1801E1ED5002E0D1
:10332000000E01D0010E176F0001F26BC7D01751CC
:103330001EE00001F25103E1DFCFF2F018D0DFCF41
:10334000E6FFF2C0E6FF70DFE552E552F3CFDEFFA5
:10335000F4CFDDFFDECF00F0DDCF01F00001800E05
:10336000011403E00101186BA9D00001F26B010107
:10337000175103E00001F25117E1DFCFF1F0000136
:10338000F151120804E30101020E186F0AD0330E46
:10339000E66E610EE66EA5EC2CF0E552E5520101F9
:1033A000186B0001F36BF46B89D017511EE000011C
:1033B000F25103E1DFCFF2F018D0DFCFE6FFF2C029
:1033C000E6FF32DFE552E552F3CFDEFFF4CFDDFF5B
:1033D000DECF00F0DDCF01F00001800E011403E02C
:1033E0000101186B6BD00001F26B0101175103E072
:1033F0000001F25162E10001F151F35D19E2020EA8
:103400000101185D09E10001F351EA6ADF0FE96E7D
:10341000000EEA22DFCFEFFF0001F32B120EF35D67
:1034200003E30101030E186FDF500001F42745D0BC
:10343000F451006E016A0050DF1803E10150DE52C2
:10344000DD180FE1020E0101185D0AE1F3C0E6FF8D
:10345000DF0EE66E000EE66E59D9E552E552E552F2
:1034600027D01C0EE66E610EE66EA5EC2CF0E55240
:10347000E552020EE66EDFCFE6FFE66A46EC2DF07F
:10348000E552E552E5520F0EE66E610EE66EA5ECD2
:103490002CF0E552E552020EE66E0001F451E66EA4
:1034A000E66A46EC2DF0E552E552E552C7EC2CF009
:1034B0000101186B020EDB5005D000D0F2D6020ECF
:1034C000DB5000D0D9CFE1FFE552E7CFD9FF1200A2
:1034D000D9CFE6FFE1CFD9FFFE0EDB50090805E3A7
:1034E000FE0EDB50300F06D005D0FE0EDB50610F14
:1034F000F60F00D0E552E7CFD9FF1200D9CFE6FF93
:10350000E1CFD9FFFE0EDB380F0BE66EE1DFE552AF
:10351000E66EF9EC2EF0E552FE0EDB500F0BE66E78
:10352000D7DFE552E66EF9EC2EF0E552E552E7CF33
:10353000D9FF1200D9CFE6FFE1CFD9FF020EE12675
:10354000DF6A010117513CE04D0EE66EF9EC2EF0FA
:10355000E552FC0EDBCFE6FFD1DFE552010EDB6A60
:10356000FC0EDB50F36E010EDBCFF4FFF350F45C86
:1035700018E2FD0EDBCFE9FFFE0EDBCFEAFFEF50D6
:10358000DF26FD0EDBCFE9FFDB2AFE0EDBCFEAFFF5
:1035900001E3DB2AEF50E66EB1DFE552010EDB2AD4
:1035A000DFD7DFCFE6FFAADFE5520D0EE66EF9ECBE
:1035B0002EF0E5520A0EE66EF9EC2EF0E55234D00C
:1035C000020EE66EF9EC2EF0E552FC0EDBCFE6FFC4
:1035D000F9EC2EF0E552010EDB6AFC0EDB50F36EC7
:1035E000010EDBCFF4FFF350F45C19E2FD0EDBCFEC
:1035F000E9FFFE0EDBCFEAFFEF50DF26FD0EDBCF4B
:10360000E9FFDB2AFE0EDBCFEAFF01E3DB2AEF5006
:10361000E66EF9EC2EF0E552010EDB2ADED7DFCFA5
:10362000E6FFF9EC2EF0E552D9CFE1FFE552E7CF06
:10363000D9FF1200D9CFE6FFE1CFD9FF0D0EE12669
:103640000C0EDF6ED950FB0FE96EFF0EDA20EA6E2A
:10365000010EEECFDBFF020EEECFDBFF030EEECF4F
:10366000DBFF040EEECFDBFF006A016A026A400E48
:10367000036ED950FB0FE96EFF0EDA20EA6EEE50B2
:103680000016EE500116EE500216EE5003160050D2
:1036900001100210031012E0F80EDBCFE6FFE66A1D
:1036A000E66AD950050FE66E000EDA20E66E4CECA5
:1036B00030F0F56E050EE15EF55016D0F80EDBCF5A
:1036C000E6FFE66AF90EDBCFE6FFFA0EDBCFE6FF98
:1036D000D950050FE66E000EDA20E66EFEEC2FF0F4
:1036E000F56E060EE15EF550F80EDB50050FE66E46
:1036F000D9CFE6FFDACFE6FF1DDFE552E552E5520E
:10370000D9CFE1FFE552E7CFD9FF1200D9CFE6FFCD
:10371000E1CFD9FF0B0EE126FC0EDB5001E1A5D273
:10372000FD0EDBCFE9FFFE0EDBCFEAFFEF500E0A06
:1037300001E198D2030A01E17DD2060A01E14BD2F0
:10374000010A01E1B1D1030A01E1ABD1010A01E1B2
:103750008ED10F0A01E157D1010A01E148D1020AD5
:1037600001E1C5D0060A50E0020A01E07ED2FC0E5B
:10377000DB50010848E2010EE76EFD0EDBCFE9FFEA
:10378000FE0EDBCFEAFFE750E926000EEA22EFCF7C
:10379000DFFFFD0EDBCFE9FFFE0EDBCFEAFF010E00
:1037A000EF6EDF5C03E3DF500C080FE2010EE76E03
:1037B000FD0EDBCFE9FFFE0EDBCFEAFFE750E92687
:1037C000000EEA220C0EEF6E0DD0010EE76EFD0E1C
:1037D000DBCFE9FFFE0EDBCFEAFFE750E926000E64
:1037E000EA22EF6A020EE66EFD0EDBCFE6FFFE0E6A
:1037F000DBCFE6FF9FDEE552E552E552DFCFE6FF85
:10380000D7EC2EF0E55231D2FC0EDB5002086EE20E
:10381000020EE76EFD0EDBCFE9FFFE0EDBCFEAFF07
:10382000E750E926000EEA22EF5010085FE3010E90
:10383000E76EFD0EDBCFE9FFFE0EDBCFEAFFE750C0
:10384000E926000EEA22EF50016A000F006E0F0E0B
:103850000122020E00C0DBFF030E01C0DBFFFD0EE4
:10386000DBCFE9FFFE0EDBCFEAFF030EEF6E020EA9
:10387000E76EFD0EDBCFE9FFFE0EDBCFEAFFE75080
:10388000E926000EEA22010EEFCFDBFFDF6A010E10
:10389000DB50DF5C1DE2020EDBCFE9FFDB2A030E0B
:1038A000DBCFEAFF01E3DB2AEF50E66E020EDF24F6
:1038B000E76EFD0EDBCFE9FFFE0EDBCFEAFFE75040
:1038C000E926000EEA22E552E750EF6EDF2ADFD745
:1038D000010EDB50020FE66EFD0EDBCFE6FFFE0EA3
:1038E000DBCFE6FF27DEE552E552E552BED1FC0E06
:1038F000DB50020801E37AD0010EE76EFD0EDBCF4C
:10390000E9FFFE0EDBCFEAFFE750E926000EEA22D0
:10391000EFCF02F0FC0EDB500224006E016A000EB5
:103920000122020E005E000E015AD8800054010EE2
:1039300001545CE3010EE76EFD0EDBCFE9FFFE0EE6
:10394000DBCFEAFFE750E926000EEA22EF50016ADA
:10395000000F006E0F0E0122040E00C0DBFF050EEB
:1039600001C0DBFFDF6AFC0EDB50FE0FDF5C1DE2F7
:10397000020EDF24E76EFD0EDBCFE9FFFE0EDBCF8C
:10398000EAFFE750E926000EEA22EF50E66E040E49
:10399000DBCFE9FFDB2A050EDBCFEAFF01E3DB2A01
:1039A000E552E750EF6EDF2ADED7FD0EDBCFE9FFF1
:1039B000FE0EDBCFEAFF050EEF6E010EE76EFD0E89
:1039C000DBCFE9FFFE0EDBCFEAFFE750E926000E72
:1039D000EA22EF6A020EE66EFD0EDBCFE6FFFE0E78
:1039E000DBCFE6FFA7DDE552E552E5523ED1070EFB
:1039F000E66EBF0EE66E430EE66E39EC24F0E5523D
:103A0000E552E55232D1FC0EDB5003082FE2030EE3
:103A1000E76EFD0EDBCFE9FFFE0EDBCFEAFFE750DE
:103A2000E926000EEA22EF50E66E020EE76EFD0E6A
:103A3000DBCFE9FFFE0EDBCFEAFFE750E926000E01
:103A4000EA22EF50E66E010EE76EFD0EDBCFE9FFD6
:103A5000FE0EDBCFEAFFE750E926000EEA22EF5028
:103A6000E66E77EC24F0E552E552E552FED0FC0E0E
:103A7000DB50010815E2010EE76EFD0EDBCFE9FF1A
:103A8000FE0EDBCFEAFFE750E926000EEA22EF50F8
:103A900002E0030E01D0040EE66E97EC24F0E5522E
:103AA000E4D0DCEC18F0E1D0FC0EDB50040801E3BC
:103AB00091D0FC0EDB500D0801E28CD0010EE76EB8
:103AC000FD0EDBCFE9FFFE0EDBCFEAFFE750E92674
:103AD000000EEA22070EEECFDBFF080EEECFDBFF73
:103AE000090EEECFDBFF0A0EEECFDBFFFC0EDB5044
:103AF000FB0FE66E050EE76EFD0EDBCF00F0FE0E4F
:103B0000DBCF01F0E7500026000E012200C0E6FFE7
:103B100001C0E6FFD950070FE96EDACFEAFFEECF1A
:103B2000E6FFEECFE6FFEECFE6FFEFCFE6FFE8ECF5
:103B300025F0F56E070EE15EF550E76E060EE7CF55
:103B4000DBFFDB5020E0070EE66E610EE66EA5ECB3
:103B50002CF0E552E552060EDB50FF0DF3CF00F0DE
:103B6000016A00BE016800C0E6FF01C0E6FFAAECE2
:103B70002DF0E552E552F10EE66E600EE66EA5EC14
:103B80002CF0E552E552FC0EDB50FB0FE66E050E05
:103B9000E76EFD0EDBCF00F0FE0EDBCF01F0E7504D
:103BA0000026000E012200C0E6FF01C0E6FFD9504A
:103BB000070FE96EDACFEAFFEECFE6FFEECFE6FFC2
:103BC000EECFE6FFEFCFE6FF74EC02F0F56E070EE6
:103BD000E15EF5504AD00001DE5117E1D5C0E6FFA5
:103BE000D60EE66E000EE66ED1C0E6FFD2C0E6FF4E
:103BF000D3C0E6FFD4C0E6FF1DDDF56E070EE15E23
:103C0000F5500001FE0EDE6F14D0FD0EDBCFE9FF94
:103C1000FE0EDBCFEAFF0C0EEF6E010EE66EFD0E20
:103C2000DBCFE6FFFE0EDBCFE6FF84DCE552E5529C
:103C3000E5521BD0FC0EDB50010813E2010EE76ECB
:103C4000FD0EDBCFE9FFFE0EDBCFEAFFE750E926F2
:103C5000000EEA22EF5002E0010E01D0000E010139
:103C6000156F03D0D4EC2FF000D0D9CFE1FFE5528F
:103C7000E7CFD9FF1200D9CFE6FFE1CFD9FF030E7E
:103C8000E126430EDF6EDE52BF0EDD6E070EF36ED1
:103C9000020EF3CFDBFF080EE66EE66AE66AFD0E63
:103CA000DBCFE6FFFE0EDBCFE6FF4CEC30F0F56E2F
:103CB000050EE15EF550FD0EDBCFE9FFFE0EDBCF1A
:103CC000EAFFEE68EE68EE68EE68010109050CE1B6
:103CD000FD0EDBCFE9FFFE0EDBCFEAFF040EE92687
:103CE000000EEA22EF680CD0FD0EDBCFE9FFFE0EDE
:103CF000DBCFEAFF040EE926000EEA22FE0EEF6E8D
:103D0000FD0EDBCFE9FFFE0EDBCFEAFF050EE92655
:103D1000000EEA22DFCFEFFFFD0EDBCFE9FFFE0E44
:103D2000DBCFEAFF060EE926000EEA22010EDBCF0A
:103D3000EFFFFD0EDBCFE9FFFE0EDBCFEAFF070E44
:103D4000E926000EEA22020EDBCFEFFFD9CFE1FF1A
:103D5000E552E7CFD9FF1200D9CFE6FFE1CFD9FF77
:103D6000080EE66EE66AC40EE66E000EE66EFD0E06
:103D7000DBCFE6FFFE0EDBCFE6FFFEEC2FF0F56EAD
:103D8000060EE15EF550000E00D0E552E7CFD9FFF8
:103D90001200D9CFE6FFE1CFD9FFE552E7CFD9FF37
:103DA0001200EB0E006E600E016E00C0F3FF01C04A
:103DB000F4FF00D01200E50E006E600E016E00C030
:0A3DC000F3FF01C0F4FF00D0120071
:063DCA001200D9CFE6FF54
:103DD000E1CFD9FFE652DF6A010109510EE189EC1A
:103DE00027F0000905E00101010E096F828203D06E
:103DF0000101020E096F010EDF6E0951020A0DE08A
:103E0000030A01E00DD00A0EE66E1BEC2EF0E5521F
:103E1000DF5002E189EC27F003D03DEC2AF000D01E
:103E2000E552E552E7CFD9FF1200D9CFE6FFE1CF47
:103E3000D9FF070EE12674EC2FF0020EF3CFDBFF63
:103E4000030EF4CFDBFF5BEC27F0F3CFDEFFF4CF04
:103E5000DDFF01010E5152E001010051DE5C006EF8
:103E60000151DD58016E040E00C0DBFF050E01C0DC
:103E7000DBFF040EDBCF00F0050EDBCF01F000010D
:103E8000800E011410E01E681F68040EDBCF23F0C3
:103E9000050EDBCF24F009EC31F0040E1CC0DBFF73
:103EA000050E1DC0DBFF040EDBCF00F0050EDBCFDF
:103EB00001F0013404E200502008000E01541EE21B
:103EC000020EDBCF1EF0030EDBCF1FF0010103510A
:103ED0001E5C026E04511F58036E130ED8800254EC
:103EE000000E03540BE2DECFE6FFDDCFE6FF61D824
:103EF000E552E552DECF00F1DDCF01F101010A51BB
:103F00000B111EE0020EDBCF1EF0030EDBCF1FF005
:103F1000010103511E5C006E04511F58016E010126
:103F200000500A5D01500B590BE2DECFE6FFDDCFFA
:103F3000E6FF3FD8E552E552DECF00F1DDCF01F1DB
:103F400001010F5111E07DEC27F0E76E060EE7CF7F
:103F5000DBFFDB500101025D07E0060EDBCF02F163
:103F600002C1E6FF60D8E55201010C510D111BE0C2
:103F7000020EDBCF1EF0030EDBCF1FF00101055157
:103F80001E5C006E06511F58016E010100500C5D51
:103F900001500D5908E27DEC27F00101026F02C1CA
:103FA000E6FF41D8E552D9CFE1FFE552E7CFD9FF8F
:103FB0001200D9CFE6FFE1CFD9FF020EE126FF0EB6
:103FC000E76EFD0EDBCF00F0FE0EDBCF01F0E75019
:103FD0000016016A0050DF6EFD0EDBCF00F0FE0E12
:103FE000DBCF01F001C000F0016A010E00C0DBFF71
:103FF000E66A020EE66ED9CFE6FFDACFE6FF040EE0
:10400000E66EBAEC15F0F56E050EE15EF55074EC57
:104010002FF0F3CF03F1F4CF04F1D9CFE1FFE55254
:10402000E7CFD9FF1200D9CFE6FFE1CFD9FFE652A3
:10403000FE0EDB50DF6EE66A010EE66ED9CFE6FFBC
:10404000DACFE6FF080EE66EBAEC15F0F56E050E57
:10405000E15EF55074EC2FF0F3CF05F1F4CF06F1EB
:10406000E552E552E7CFD9FF1200D9CFE6FFE1CF05
:10407000D9FFE552E7CFD9FF1200D9CFE6FFE1CF54
:10408000D9FF0F0EE126FE0EDB500A0A01E155D1E1
:10409000030A01E151D10E0A01E148D1010A01E10F
:1040A00044D1030A23E0060A13E0010A01E0ACD27E
:1040B000FB0EDB5000080BE2FC0EDBCFE9FFFD0E30
:1040C000DBCFEAFFEF50E66E50EC27F0E5529CD2D2
:1040D0005BEC27F0F3CF00F0F4CF01F000C0E6FF77
:1040E00001C0E6FF66DFE552E5528ED2FB0EDB50E3
:1040F00001E18AD2FC0EDBCFE9FFFD0EDBCFEAFF48
:10410000EF50050A01E1CDD0010A01E1AED0070A66
:1041100001E18FD0010A48E0030A01E005D1030E56
:10412000F36EFB0EDBCFF4FFF350F45C3CE3020EC6
:10413000E76EFC0EDBCFE9FFFD0EDBCFEAFFE750B9
:10414000E926000EEA22EFCF02F002C003F0026A75
:10415000010EE76EFC0EDBCFE9FFFD0EDBCFEAFFC1
:10416000E750E926000EEA22EF5000010224006E1B
:10417000000E0320016E00C0E6FF01C0E6FF7AECEE
:104180002FF0E552E552F3CF0AF1F4CF0BF174ECC6
:104190002FF001010A51F35C0101036F01010B5182
:1041A000F4580101046FC0D0030EF36EFB0EDBCF99
:1041B000F4FFF350F45C3CE3020EE76EFC0EDBCF41
:1041C000E9FFFD0EDBCFEAFFE750E926000EEA2209
:1041D000EFCF02F002C003F0026A010EE76EFC0EA0
:1041E000DBCFE9FFFD0EDBCFEAFFE750E926000E4B
:1041F000EA22EF5000010224006E000E0320016E3F
:1042000000C0E6FF01C0E6FF7AEC2FF0E552E55270
:10421000F3CF0CF1F4CF0DF174EC2FF001010C5140
:10422000F35C0101056F01010D51F4580101066FA6
:104230007BD0020EF36EFB0EDBCFF4FFF350F45C89
:1042400013E3010EE76EFC0EDBCFE9FFFD0EDBCFC3
:10425000EAFFE750E926000EEA22EF5002E0010EE5
:1042600001D0000E01010E6F5FD0020EF36EFB0E47
:10427000DBCFF4FFF350F45C13E3010EE76EFC0EAA
:10428000DBCFE9FFFD0EDBCFEAFFE750E926000EAA
:10429000EA22EF5002E0010E01D0000E01010F6F83
:1042A00043D0020E0101095D3EE1040EF36EFB0EE8
:1042B000DBCFF4FFF350F45C36E3010EE76EFC0E47
:1042C000DBCFE9FFFD0EDBCFEAFFE750E926000E6A
:1042D000EA22EF5002E0010E01D0000E106F030E33
:1042E000E76EFC0EDBCFE9FFFD0EDBCFEAFFE75008
:1042F000E926000EEA22EFCF00F000C001F0006ACC
:10430000020EE76EFC0EDBCFE9FFFD0EDBCFEAFF0E
:10431000E750E926000EEA22EF5001010024076F62
:10432000000E0120086F00D06FD16ED17DEC27F018
:10433000E66E79DEE55268D167D10C0EDB6A0101C9
:10434000090508E1030EF36EFB0EDBCFF4FFF3501B
:10435000F45C01E259D1020EE76EFC0EDBCFE9FFFF
:10436000FD0EDBCFEAFFE750E926000EEA22EFCF91
:1043700002F002C003F0026A010EE76EFC0EDBCF12
:10438000E9FFFD0EDBCFEAFFE750E926000EEA2247
:10439000EF5000010224006E000E0320016EFF0E9C
:1043A00000167F0E011600C0DEFF01C0DDFF4EECDF
:1043B00028F0F3CF00F0F4CF01F00050011001E03D
:1043C00023D1FC0EDBCFE9FFFD0EDBCFEAFFEF5080
:1043D00071E0010A01E017D10A0EDB6AFB0EDB5027
:1043E000FD0FF36E0A0EDBCFF4FFF350F45C35E201
:1043F0000A0EDB50030FE76EFC0EDBCFE9FFFD0E6C
:10440000DBCFEAFFE750E926000EEA22EF50E66E26
:104410000A0EDB50E76E000EDFCF02F0010EDBCF9D
:1044200003F0E7500226000E032202C0E6FF03C09D
:10443000E6FFB3EC28F0E552E552E552F3CF00F089
:10444000F4CF01F00050011005E0010EF36E0C0EE8
:10445000F3CFDBFF0A0EDB2AC1D7020EE76EFC0E9C
:10446000DBCFE9FFFD0EDBCFEAFFE750E926000EC8
:10447000EA22EF50800B01E1C6D0FB0EDB50FD0FAE
:10448000E66E030EE76EFC0EDBCFE9FFFD0EDBCF21
:10449000EAFFE750E926000EEA22E552E750EF6E08
:1044A0004EEC28F0F3CF00F0F4CF01F000500110F3
:1044B00001E0A9D0010EE76EFC0EDBCFE9FFFD0E97
:1044C000DBCFEAFFE750E926000EEA22020EEFCF2B
:1044D000DBFFE76EFC0EDBCFE9FFFD0EDBCFEAFF73
:1044E000E750E926000EEA22030EEFCFDBFFE76E6E
:1044F000FC0EDBCFE9FFFD0EDBCFEAFFE750E9263C
:10450000000EEA220B0EEFCFDBFFDB50060805E2C0
:10451000060EF36E0B0EF3CFDBFF0A0EDB6A0B0EFB
:10452000DB50F36E0A0EDBCFF4FFF350F45C42E293
:104530000A0EDB50E76E000EDFCF00F0010EDBCF7E
:1045400001F0E7500026000E012200C0E6FF01C086
:10455000E6FFA5EC27F0E552E5520D0EF3CFDBFFA9
:104560000E0EF4CFDBFF0D0EDBCF00F00E0EDBCF17
:1045700001F00001800E011409E0010EF36E0C0E33
:10458000F3CFDBFF0D0EDB6A0E0EDB6AD950020F94
:10459000006EDACF01F00A0EDB50020F0F0100248B
:1045A000E96E000E0120EA6E0D0EDBCFEFFF0A0E62
:1045B000DB2AB5D70C0EDB5012E0E66A020EE66E7F
:1045C000D950020FE66E000EDA20E66E0B0EE66E94
:1045D000BAEC15F0F56E050EE15EF55013D0E66A03
:1045E0000B0EDB50020FE66ED950020FE66E000E86
:1045F000DA20E66E0B0EE66EBAEC15F0F56E050EDF
:10460000E15EF55000D000D0D9CFE1FFE552E7CF11
:10461000D9FF1200D9CFE6FFE1CFD9FFFE0EDB5064
:10462000050811E1FB0EDBCFE6FFFC0EDBCFE6FF5A
:10463000FD0EDBCFE6FFFE0EDBCFE6FF1EDDE55213
:10464000E552E552E552E552E7CFD9FF1200D9CF46
:10465000E6FFE1CFD9FFE552E7CFD9FF1200D9CF6E
:10466000E6FFE1CFD9FF030EE126020E0101095D4D
:1046700001E0ECD0105101E1E9D04FEC00F000096D
:1046800001E1E4D0006A016A026A400E036ED9506B
:10469000FB0FE96EFF0EDA20EA6EEE500016EE50C8
:1046A0000116EE500216EE500316005001100210D3
:1046B000031002E1000E01D0010EE76E020EE7CFFB
:1046C000DBFFD950FB0FE96EFF0EDA20EA6EEE52E7
:1046D000EE52EE521F0EEE1607C100F008C101F0B7
:1046E000026A036AD950FB0FE96EFF0EDA20EA6E08
:1046F0000050EE5C0150EE580250EE580350EE5858
:1047000001E2A4D0400E0101056A0725046E08519C
:104710000522066A076AD950FB0FE96EFF0EDA2000
:10472000EA6E0450EE5C0550EE580650EE58075005
:10473000EE5801E38BD007C104F008C105F0066A0A
:10474000076AD950FB0FE96EFF0EDA20EA6E0450BB
:10475000EE5C006E0550EE58016E0650EE58026E8B
:104760000750EE58036E010E00C0DBFFDBCFE6FF03
:104770000AEC2BF0E552F36EFA0EDB50F35C01E02D
:1047800065D0020EDB5054E0FA0EDBCFE6FFF80EE8
:10479000DBCFE6FFF90EDBCFE6FF010EDB500101B8
:1047A000016A0725006E08510122026A036A00C0EF
:1047B000E6FF01C0E6FF02C0E6FF03C0E6FFE8EC4B
:1047C00025F0F56E070EE15EF550F80EDBCFE6FF43
:1047D000F90EDBCFE6FF010EDBCFE6FFE8EC2BF0B6
:1047E000E552E552E552DF6EDF5021E1FA0EDBCFF4
:1047F000E6FFF80EDBCFE6FFF90EDBCFE6FF010E9A
:10480000DB500101016A0725006E08510122026A8E
:10481000036A00C0E6FF01C0E6FF02C0E6FF03C076
:10482000E6FFE8EC25F0F56E070EE15EF5500ED0E0
:10483000F80EDBCFE6FFF90EDBCFE6FF010EDBCF94
:10484000E6FF64EC2BF0E552E552E552D9CFE1FFEB
:10485000E552E7CFD9FF1200D9CFE6FFE1CFD9FF6C
:0C486000010E00D0E552E7CFD9FF120096
:04486C001200120024
:104870001200D9CFE6FFE1CFD9FFE652800E6F6E6E
:10488000E00E6E14800801E0FBD7E00E736E0F019E
:10489000406B306B206B640E606E600E506FA46ACC
:1048A000030EA36EA56E1A6B1B6B186B196B016B55
:1048B0001E6B1F6B1C6B1D6B080E056FFC0EDBCF98
:1048C000E6FFFD0EDBCFE6FFFE0EDBCFE6FF0FD8E7
:1048D000E552E552E552DF6E010EE66E28D8E5524C
:1048E000DF5000D0E552E552E7CFD9FF1200D9CF13
:1048F000E6FFE1CFD9FFE6526F50DF6E800E6F6E9C
:10490000E00E6E14800801E0FBD7FE0EDB50706EE7
:10491000FD0EDB50716EFC0EDB50726EDF506F6E61
:10492000000E00D0E552E552E7CFD9FF1200D9CFF3
:10493000E6FFE1CFD9FFE652FE0EDB50040803E1AB
:10494000200EDF6E07D0FE0EDB0403E1600EDF6E8B
:1049500001D0DF6ADF506F6EE00E6E14006EDF5024
:10496000005C01E0F9D7E552E552E7CFD9FF12002C
:10497000A36A300E6F6E1200D9CFE6FFE1CFD9FFE8
:10498000E6526F50DF6EFE0EDB5005E0F10E6F1445
:104990000A096F6E04D0F10E6F140C096F6E60AED1
:1049A00017D0E00E0F0142150101D8801D550101FD
:1049B000206F20510DE11F510F01415D09E1609E03
:1049C000FE0EDB5002E0A49201D0A49001011D690B
:1049D000DF506F6EE552E552E7CFD9FF1200D9CF15
:1049E000E6FFE1CFD9FFE652FE0EDF6E01011C515A
:1049F00006E0F10E6F140A096F6EDF6A06D0F10E41
:104A00006F140C096F6E60BEDF6ADF5001E0D9D011
:104A10000F0E6514E66EF90EDBCFE9FFFA0EDBCF61
:104A2000EAFFE552E750EF6E080EE66EE66A660EA4
:104A3000E66E0F0EE66EFB0EDBCFE6FFFC0EDBCF65
:104A4000E6FFFEEC2FF0F56E060EE15EF55062A675
:104A500078D06450046E056A066A076A6350086E6F
:104A6000096A0A6A0B6A080E1F0B07E0D89008361D
:104A700009360A360B36E806F9E1085004260950D3
:104A800005220A5006220B500722030E62140C6EF8
:104A90000D6A0E6A0F6A100E1F0B07E0D8900C36D5
:104AA0000D360E360F36E806F9E10C5004260D508F
:104AB00005220E5006220F500722E00E6214106EDF
:104AC000116A126A136A0D0E1F0B07E0D890103698
:104AD000113612361336E806F9E11050042611504B
:104AE000052212500622135007226150146E156AD7
:104AF000166A176A150E1F0B07E0D8901436153684
:104B000016361736E806F9E104501424006E0550F5
:104B10001520016E06501620026E07501720036EF6
:104B2000800E0326FD0EDBCFE9FFFE0EDBCFEAFF92
:104B300000C0EEFF01C0EEFF02C0EEFF03C0EEFFBB
:104B400023D06150046E056A030ED89004360536F2
:104B5000E804FBE16250E00BE838E840000104247F
:104B6000006E000E0520016E026A036AFD0EDBCFA7
:104B7000E9FFFE0EDBCFEAFF00C0EEFF01C0EEFF53
:104B800002C0EEFF03C0EEFF60A60AD0FD0EDBCF31
:104B9000E9FFFE0EDBCFEAFFEE52EE52EE52EE8C54
:104BA000609E01011C5102E0A49201D0A4901C510E
:104BB00002E01C6B06D00F0150AF03D00101010EC3
:104BC0001C6FDF5000D0E552E552E7CFD9FF12004D
:104BD000D9CFE6FFE1CFD9FF040EE126A00E6E1477
:104BE00002E0F80E45D1F10E6F1408096F6E0F0147
:104BF00040A708D001011E5102E1FA0E39D10F0180
:104C000040B7FDD7006A016A026A800E036ED95070
:104C1000FB0FE96EFF0EDA20EA6EEE500016EE5042
:104C20000116EE500216EE5003160050011002104D
:104C3000031001E17FD0FB0EDBCF44FFDBCF00F0A0
:104C4000FC0EDBCF01F0FD0EDBCF02F0FE0EDBCF62
:104C500003F0080ED8900332023201320032E80627
:104C6000F9E100C043FFFB0EDBCF08F0FC0EDBCF09
:104C700009F0FD0EDBCF0AF0FE0EDBCF0BF00AC011
:104C800004F00BC005F00001066A076A030E041663
:104C9000056A066A076AFB0EDBCF0CF0FC0EDBCF61
:104CA0000DF0FD0EDBCF0EF0FE0EDBCF0FF00D0E84
:104CB000D8900F320E320D320C32E806F9E1E00ED8
:104CC000106E116A126A136A10500C1611500D16EC
:104CD00012500E1613500F1604500C24006E05507F
:104CE0000D20016E06500E20026E07500F20036E3D
:104CF000080E0026000E01220222032200C042FFFD
:104D0000FB0EDBCF00F0FC0EDBCF01F0FD0EDBCFA6
:104D100002F0FE0EDBCF03F0150ED8900332023204
:104D200001320032E806F9E100C041FF030E42CF34
:104D3000DBFF38D0070E006E016A026A036AD950A1
:104D4000FB0FE96EFF0EDA20EA6EEE500016EE5011
:104D50000116EE500216EE500316050E1F0B07E06B
:104D6000D8900036013602360336E806F9E1030E24
:104D700000C0DBFFDBCF42FFFB0EDBCF00F0FC0E01
:104D8000DBCF01F0FD0EDBCF02F0FE0EDBCF03F038
:104D9000030ED8900332023201320032E806F9E104
:104DA00000C041FFF80EDB50080805E2080EF36E64
:104DB000F80EF3CFDBFFF80EDB50DF6E006A016AFE
:104DC000026A400E036ED950FB0FE96EFF0EDA2027
:104DD000EA6EEE500016EE500116EE500216EE503E
:104DE0000316005001100210031002E0F80EDB8CD5
:104DF000F80EDBCF45FFD950010FE96EDACFEAFF9D
:104E0000460EEE6E0F0EED6EDF50DF0600091EE05F
:104E1000030EDB500F01425D01E028DDF90EDBCF10
:104E2000E9FFDB2AFA0EDBCFEAFF01E3DB2AEF50D2
:104E3000E66E010EDBCFE9FFDB2A020EDBCFEAFFD5
:104E400001E3DB2AE552E750EF6EDED7030EDB50BD
:104E50000F01425D01E00ADDE00E0F014215010184
:104E60001D6F41CF1FF10F010B0E406F000E00D0E0
:0C4E7000D9CFE1FFE552E7CFD9FF1200D7
:044E7C009698836A17
:104E8000956AF80E936E800E946E82908292829450
:104E9000A00EC26EC20EC16EC280C2848280120099
:104EA000D9CFE6FFE1CFD9FFFE0EDB50836EE5528E
:104EB000E7CFD9FF1200D9CFE6FFE1CFD9FF020E2D
:104EC000E126C350DF6E010EC4CFDBFFC350DF5CB1
:104ED00003E1C2B403D001D0F4D7C284DECF00F026
:104EE000DDCF01F000C0F3FF01C0F4FF00D0D9CF47
:104EF000E1FFE552E7CFD9FF1200811CE8380F0B24
:104F0000030B00D01200020EE66EE2EC32F0E55226
:104F100012000D0EC86EE66A080EE66E76EC32F0F0
:104F2000E552E552000EE66EE66A0FD8E552E5520C
:104F3000F3CF00F0F4CF01F00001800E011402E184
:104F4000010E01D0000E00D01200D9CFE6FFE1CF54
:104F5000D9FFE652FD0EDBCF00F0FE0EDBCF01F0F5
:104F6000070ED89001320032E804FBE10E0E001467
:104F7000DF6EA196C750040B01E0010E006E1F0EFC
:104F8000C514001001E0F6D7C580C5B0FED7A1A6B4
:104F900003D0F368F4687DD0A00EDF24E66E91ECB8
:104FA00032F0E552000904E0FD0EF36EF46871D0B2
:104FB000C750040B01E0010E006E1F0EC514001057
:104FC00001E0F6D7C5AC04D0FE0EF36EF46861D0F4
:104FD000FF0EE76EFD0EDBCF00F0FE0EDBCF01F023
:104FE000E7500016016A0050E66E91EC32F0E5528F
:104FF000000904E0FD0EF36EF4684BD0C750040BBB
:1050000001E0010E006E1F0EC514001001E0F6D77E
:10501000C5AC04D0FE0EF36EF4683BD0C582C5B2B9
:10502000FED7A1A603D0F368F46833D0A10EDF2425
:10503000E66E91EC32F0E552000904E0FD0EF36EED
:10504000F46827D0C750040B01E0010E006E1F0E5C
:10505000C514001001E0F6D7C5AC04D0FE0EF36E07
:10506000F46817D0C586C5B6FED7C58AC588C5B849
:10507000FED7C584C5B4FED7A1A603D0F368F468F3
:1050800008D0C950006E016A00C0F3FF01C0F4FFF0
:1050900000D0E552E552E7CFD9FF1200D9CFE6FFA5
:1050A000E1CFD9FFE652DF6AA196C750040B01E0B9
:1050B000010E006E1F0EC514001001E0F6D7C5806A
:1050C000C5B0FED7A1A603D0F368F46847D0A00E00
:1050D000DF24E66E91EC32F0E552000904E0FD0EAB
:1050E000F36EF4683BD0C750040B01E0010E006E74
:1050F0001F0EC514001001E0F6D7A1A603D0F36877
:10510000F4682CD0C5AC1FD0C582C5B2FED7A1A60D
:1051100003D0F368F46822D0A00EDF24E66E91EC91
:1051200032F0E552000904E0FD0EF36EF46816D08B
:10513000C750040B01E0010E006E1F0EC5140010D5
:1051400001E0F6D7DFD7C584C5B4FED7A1A603D04A
:10515000F368F46803D0F36AF46A00D0E552E552CC
:10516000E7CFD9FF1200D9CFE6FFE1CFD9FF030E79
:10517000E126FD0EDBCF00F0FE0EDBCF01F0070EC7
:10518000D89001320032E804FBE10E0E0014DF6E0D
:10519000010EDB6A020EDB6A81DFDE52F3CFDEFF37
:1051A000F4CFDDFFDD52D950010FE96EDACFEAFF0F
:1051B000EE50ED100BE0010EDBCF00F0020EDBCF66
:1051C00001F000C0F3FF01C0F4FF76D0A196C750F4
:1051D000040B01E0010E006E1F0EC514001001E06B
:1051E000F6D7C580C5B0FED7A1A603D0F368F46892
:1051F00063D0A00EDF24E66E91EC32F0E552000998
:1052000004E0FD0EF36EF46857D0C750040B01E0C4
:10521000010E006E1F0EC514001001E0F6D7C5ACDC
:1052200004D0FE0EF36EF46847D0FF0EE76EFD0E5D
:10523000DBCF00F0FE0EDBCF01F0E7500016016A75
:105240000050E66E91EC32F0E552000904E0FD0EEC
:10525000F36EF46831D0C750040B01E0010E006E0C
:105260001F0EC514001001E0F6D7C5AC04D0FE0E29
:10527000F36EF46821D0FC0EDBCFE6FF91EC32F048
:10528000E552000904E0FD0EF36EF46815D0C75036
:10529000040B01E0010E006E1F0EC514001001E0AA
:1052A000F6D7C584C5B4FED7A1A603D0F368F468C9
:1052B00003D0F36AF46A00D0D9CFE1FFE552E7CF1B
:1052C000D9FF1200D9CFE6FFE1CFD9FF030EE126C7
:1052D000FD0EDBCF00F0FE0EDBCF01F0070ED89005
:1052E00001320032E804FBE10E0E0014DF6E010E05
:1052F000DB6A020EDB6AF90EDBCF00F0FA0EDBCFC1
:1053000001F0013404E200502008000E015404E2D0
:10531000FC0EF36EF468ABD0C1DEDE52F3CFDEFFDD
:10532000F4CFDDFFDD52D950010FE96EDACFEAFF8D
:10533000EE50ED100BE0010EDBCF00F0020EDBCFE4
:1053400001F000C0F3FF01C0F4FF91D0A196C75057
:10535000040B01E0010E006E1F0EC514001001E0E9
:10536000F6D7C580C5B0FED7A1A603D0F368F46810
:105370007ED0A00EDF24E66E91EC32F0E5520009FB
:1053800004E0FD0EF36EF46872D0C750040B01E028
:10539000010E006E1F0EC514001001E0F6D7C5AC5B
:1053A00004D0FE0EF36EF46862D0FF0EE76EFD0EC1
:1053B000DBCF00F0FE0EDBCF01F0E7500016016AF4
:1053C0000050E66E91EC32F0E552000904E0FD0E6B
:1053D000F36EF4684CD0C750040B01E0010E006E70
:1053E0001F0EC514001001E0F6D7C5AC04D0FE0EA8
:1053F000F36EF4683CD0F90EDBCF00F0DB06FA0E5A
:10540000DBCF01F001E2DB060050011025E0FB0ECE
:10541000DBCFE9FFDB2AFC0EDBCFEAFF01E3DB2A6F
:10542000EF50E66E91EC32F0E552000904E0FD0E1B
:10543000F36EF4681CD0C750040B01E0010E006E3F
:105440001F0EC514001001E0F6D7C5AC04D0FE0E47
:10545000F36EF4680CD0CFD7C584C5B4FED7A1A62F
:1054600003D0F368F46803D0F36AF46A00D0D9CFAC
:0A547000E1FFE552E7CFD9FF12007B
:06547A001E0EE66EE66A5C
:105480002C0EE66EBDEC31F0E552E552E552000E11
:1054900000D01200ACA2FED71200ABA202D0AB9893
:1054A000AB889EAA03D038EC32F0F7D700D01200B8
:1054B000D9CFE6FFE1CFD9FF020EE126EBDF57ECB3
:1054C00032F0F3CFDEFFF4CFDDFFDECF02F0DDCF31
:1054D00003F002C0E6FF03C0E6FF57EC32F0E552EE
:1054E000E7CF03F0E552E7CF02F00250F35C006E25
:1054F0000350F458016EFE0EDB50046E056A710E07
:105500000502F3CF05F0020E0402F3500526710EDA
:105510000402F3CF04F0F45005260450005C05505B
:10552000015801E2D2D7D9CFE1FFE552E7CFD9FF49
:105530001200D9CFE6FFE1CFD9FFACA2FED7FE0E15
:10554000DBCFE6FFA9EC32F0E552E552E7CFD9FF19
:105550001200D9CFE6FFE1CFD9FF020EE126FE0E01
:10556000DB9CDB9E97DF2C0EAF6EE66AE2DFE55236
:1055700091DF070EE66E9CDFE5521E0EAF6E550EF4
:10558000E66ED7DFE552FE0EDB50DF6E010EDB6A02
:10559000FE0EDBA002D0010EDB2AFE0EDBA202D043
:1055A000010EDB2AFE0EDBA402D0010EDB2AFE0E6A
:1055B000DBA802D0010EDB2A010EDBB0DF8CDE524D
:1055C000DD6EFE0EDBA202D0010EDB2AFE0EDBA694
:1055D00002D0010EDB2AFE0EDBA802D0010EDB2A70
:1055E000FE0EDBAA02D0010EDB2A010EDBB0DF8E3D
:1055F000070EE66E5DDFE552DFCFE6FF9ADFE5528C
:10560000020EE66E55DFE552D9CFE1FFE552E7CF56
:10561000D9FF1200D9CFE6FFE1CFD9FFE652FE0E47
:10562000DB380F0B030B006E010E005204E0E8465E
:10563000FE0B0006FCE1DF6EDF0402E1020EDF6E0E
:10564000DF5000D0E552E552E7CFD9FF1200D9CFA5
:10565000E6FFE1CFD9FFFE0EDB98DB9ADB9CDB9EF9
:10566000FD0EDB50080A1EE00C0A11E0070A04E0F8
:10567000010A01E000D021D0100E006EFE0EDBCF3B
:10568000E7FF0050E726FE0EE7CFDBFF16D0200E27
:10569000006EFE0EDBCFE7FF0050E726FE0EE7CFE1
:1056A000DBFF0BD0300E006EFE0EDBCFE7FF0050AD
:1056B000E726FE0EE7CFDBFF00D0FE0EDB5000D06A
:1056C000E552E7CFD9FF1200D9CFE6FFE1CFD9FFEE
:1056D000040EE126FE0EDB9CDB9EDBCFE6FF39DF0E
:1056E000E552FE0EDBCFE6FF95DFE552DF6E020EE0
:1056F000DB6A030EDB6A010EDB6ADF50F36E010E1C
:10570000DBCFF4FFF350F45C52E2010EDB50E76EA6
:10571000FC0EDBCFE9FFFD0EDBCFEAFFE750E92609
:10572000000EEA22EF50006E016AD950020FE96EB6
:10573000DACFEAFF0050EE260150ED22020EDBCF59
:1057400000F0030EDBCF01F0000E005C010E0158EB
:1057500016E3010EE76E020EDBCF00F0030EDBCF87
:1057600001F0E7500026000E0122FF0E0016000E89
:105770000116020E00C0DBFF030E01C0DBFF020EAC
:10578000E66E96DEE552010EDB50E76EFC0EDBCFD7
:10579000E9FFFD0EDBCFEAFFE750E926000EEA2223
:1057A000EF50E66EC6DEE552010EDB2AA6D7020EEA
:1057B000E66E7EDEE552020EDB1CE66EBADEE552D8
:1057C000000E00D0D9CFE1FFE552E7CFD9FF12009C
:1057D000D9CFE6FFE1CFD9FF060EE1265EDEFE0E51
:1057E000DBCFE6FFB6DEE55258DEFE0EDBCFE6FF8E
:1057F00011DFE552E76E010EE7CFDBFFDF6A010E36
:10580000DB28DF5C45E274EC2FF0020EF3CFDBFF08
:10581000030EF4CFDBFF9EBA23D0ABA202D0AB982D
:10582000AB8874EC2FF0040EF3CFDBFF050EF4CF42
:10583000DBFF040EDBCF02F0050EDBCF03F0020E20
:10584000DB50025C006E030EDB500358016E090E44
:10585000D8800054000E015402E2070E4CD0DBD772
:1058600038EC32F00101196F010EDB50DF5C0EE203
:10587000DF50E76EFC0EDBCFE9FFFD0EDBCFEAFF6A
:10588000E750E926000EEA2219C1EFFFDF2AB7D759
:1058900001011A6B1B6BDF6A010EDB50DF5C24E237
:1058A000DF50E76EFC0EDBCFE9FFFD0EDBCFEAFF3A
:1058B000E750E926000EEA22EF50006E016A005020
:1058C0001A2701501B23000E1A5D010E1B590AE313
:1058D000010E1A251A6F000E1B211B6FFF0E1A17DF
:1058E000000E1B17DF2AD8D71A1D195D02E0060E1D
:1058F00002D0000E00D0D9CFE1FFE552E7CFD9FFAB
:0E59000012004F0EAB16AC9ACF0E9D16120081
:02590E00000E89
:1059100000D01200D9CFE6FFE1CFD9FFC9EC2EF0BD
:1059200000090FE0FE0EDBCFE6FFF9EC2EF0E552AA
:10593000FE0EDB500A0805E10D0EE66EF9EC2EF0C6
:10594000E552E552E7CFD9FF1200D9CFE6FFE1CF0C
:10595000D9FFFD0EDBCFF6FFFE0EDBCFF7FF080011
:10596000F55011E0FD0EDBCFF6FFFE0EDBCFF7FFAB
:105970000800F550E66ECEDFE552FD0EDB2AFE0E86
:1059800001E3DB2AE6D7E552E7CFD9FF12000A0E82
:10599000E66EC0DFE5521200D9CFE6FFE1CFD9FFB6
:1059A000060EE126D9CF00F0DACF01F0040E00C0D8
:1059B000DBFF050E01C0DBFF0F0EE76EFD0EDBCF38
:1059C00000F0FE0EDBCF01F0E7500016016A300E4A
:1059D0000026000E0122040EDBCFE9FF050EDBCF0F
:1059E000EAFF00C0EFFF040EDBCFE9FF050EDBCFBF
:1059F000EAFFEF5039080AE2270E006E040EDBCFF3
:105A0000E9FF050EDBCFEAFF0050EF26040EDB2A8C
:105A1000050E01E3DB2AD950FD0FE96EFF0EDA20F7
:105A2000EA6E040E0F0B06E0EC52D890ED32EF3226
:105A3000E806FAE1D950FD0FE96EFF0EDA20EA6EB2
:105A4000EE50ED10B9E1040EDB06DBCF00F0050EE1
:105A500001E2DB06DBCF01F0D9CF02F0DACF03F0B1
:105A60000250005C035001580BE3040EDBCFE9FF4A
:105A7000050EDBCFEAFFEF50E66E4CDFE552E3D7D1
:105A8000D9CFE1FFE552E7CFD9FF1200D9CFE6FF2A
:105A9000E1CFD9FF020EE126FD0EDBCFDEFFDBCF2B
:105AA000DDFFD9CFE9FFDACFEAFF040E0F0B06E0E6
:105AB000EC52D890ED32EF32E806FAE1FC0EDB064C
:105AC000FC0EDBCF00F0000EE76E0018E8AE02D04F
:105AD000003403D0E750D880005417E2D9CFE9FF53
:105AE000DACFEAFFEE50ED1010E0FC0EDB06D9CF66
:105AF000E9FFDACFEAFF040E0F0B06E0EC52D89074
:105B0000ED32EF32E806FAE1DBD7FC0EDBCFF3FF34
:105B1000DB06F350006E000EE76E0018E8AE02D010
:105B2000003403D0E750D880005405E2300EE66E12
:105B3000F1DEE552EAD7FD0EDBCFE6FFFE0EDBCF4E
:105B4000E6FF2ADFE552E552D9CFE1FFE552E7CF84
:105B5000D9FF1200D9CFE6FFE1CFD9FF070EE1262A
:105B6000D9CF00F0DACF01F0050E00C0DBFF060E42
:105B700001C0DBFFFD0EDBCF00F0FE0EDBCF01F03E
:105B80000A0E236E246A00C01EF001C01FF0C0EC94
:105B900032F01AC000F01BC001F0300E0026000EDB
:105BA0000122050EDBCFE9FFDB2A060EDBCFEAFF81
:105BB00001E3DB2A00C0EFFFD950FD0FE96EFF0EB5
:105BC000DA20EA6E0A0E236E246AEECF1EF0EDCFC5
:105BD0001FF0C0EC32F01EC0EEFF1FC0EDFFD95029
:105BE000FD0FE96EFF0EDA20EA6EEE50ED10C2E115
:105BF000050EDB06DBCF00F0060E01E2DB06DBCF95
:105C000001F0D9CF02F0DACF03F00250005C03506C
:105C100001580BE3050EDBCFE9FF060EDBCFEAFFF1
:105C2000EF50E66E77DEE552E3D7D9CFE1FFE552DC
:065C3000E7CFD9FF1200CE
:0A5C3600D9CFE6FFE1CFD9FF050E3C
:105C4000E126010E046E056A066A076AFE0EDB0491
:105C50001F0B04C000F005C001F006C002F007C031
:105C600003F007E0D8900036013602360336E80626
:105C7000F9E14B0E216E226A236A246A00C01CF0EF
:105C800001C01DF002C01EF003C01FF085EC31F012
:105C900018C000F019C001F01AC002F01BC003F0D8
:105CA000010E00C0DBFF020E01C0DBFF030E02C0CD
:105CB000DBFF040E03C0DBFF010EDBCF04F0020E9E
:105CC000DBCF05F0030EDBCF06F0040EDBCF07F0D1
:105CD000020E216E226A236A246A04C01CF005C0E9
:105CE0001DF006C01EF007C01FF0D5EC30F01CC040
:105CF00004F01DC005F01EC006F01FC007F0D00E56
:105D00000426120E0522130E0622000E072204C0DE
:105D10001CF005C01DF006C01EF007C01FF0010EEC
:105D2000DBCF21F0020EDBCF22F0030EDBCF23F01E
:105D3000040EDBCF24F0D5EC30F01CC000F01DC009
:105D400001F01EC002F01FC003F00006000E015A51
:105D5000025A035A0050DF6EDFCF00F0016A00BE26
:105D6000016800C0E6FF01C0E6FF3C0EE66EBDEC38
:105D700031F0E552E552E552948E949C0101010EFA
:105D8000216F000E00D0D9CFE1FFE552E7CFD9FF58
:105D900012000101215100D01200ACA2FED7010176
:105DA000216B4F0EAB16AC9ACF0E9D161200D9CFB9
:105DB000E6FFE1CFD9FFF1DFFE0EDBCFE6FF3BDFF1
:105DC000E55200D0E552E7CFD9FF12009EAA09D0D4
:105DD00038EC32F0006E016A00C0F3FF01C0F4FF3E
:105DE00007D0ABA202D0AB98AB88F368F46800D0C0
:105DF0001200D9CFE6FFE1CFD9FFACA2FED7FE0E4D
:105E0000DBCFE6FFA9EC32F0E552E552E7CFD9FF50
:025E100012007E
:0E5E1200C00EF26E0A0ED06EA082A2820101B6
:105E2000116B126BCD0EE66E15EC32F0E5521200DE
:105E3000DACFE4FFE2CFDAFFE9CFE4FFEACFE4FF15
:105E400000EE00F0180EE80403E3EECFE4FFFBD70A
:105E5000E652E55200EE17F0180EE80403E3E5CF32
:105E6000EDFFFBD7E5CFEAFFE5CFE9FFE5CFDAFFAE
:105E70001100DACFE4FFE2CFDAFFE9CFE4FFEACFA7
:105E8000E4FF00EE00F0180EE80403E3EECFE4FFB9
:105E9000FBD7E652A050020B08E0A150020B05E030
:105EA0000101112B000E1223A192A4A005D0E66AD5
:105EB000BCEC24F0E552A490A4A206D0010EE66E3C
:105EC000BCEC24F0E552A492E55200EE17F0180E57
:105ED000E80403E3E5CFEDFFFBD7E5CFEAFFE5CF2D
:105EE000E9FFE5CFDAFF110011C1F3FF12C1F4FFA2
:105EF00000D01200D9CFE6FFE1CFD9FF050EE76E43
:105F0000FD0EDBCF00F0FE0EDBCF01F0E7500026E8
:105F1000000E01220A0E236E246A00C01EF001C08A
:105F20001FF0C0EC32F01EC000F01FC001F000C036
:105F3000F3FF01C0F4FF00D0E552E7CFD9FF120014
:105F4000D9CFE6FFE1CFD9FF020EE126CDDFF3CFB7
:105F5000DEFFF4CFDDFFDECF02F0DDCF03F002C0C5
:105F6000E6FF03C0E6FFC0DFE552E7CF03F0E552EE
:105F7000E7CF02F00250F35C006E0350F458016E5C
:105F8000FD0EDBCF04F0FE0EDBCF05F00450005C0D
:105F90000550015802E207D8DED7D9CFE1FFE5521C
:0A5FA000E7CFD9FF12001200120033
:065FAA00D9CFE6FFDACFBB
:105FB000E6FFFA0EE3CFD9FFFB0EE3CFDAFFFC0ECC
:105FC000E3CFE9FFFD0EE3CFEAFFF80EE35003E174
:105FD000F90EE35008E0F80EE30602E2F90EE306DC
:105FE000DE50EE5CF2E0F36EFF0EE3CFDAFFE55237
:105FF000FF0EE3CFD9FFE552F3501200D9CFE6FFF1
:10600000DACFE6FFFA0EE3CFD9FFFB0EE3CFDAFFDC
:10601000FC0EE3CFE9FFFD0EE3CFEAFFE9CFF3FF8C
:10602000EACFF4FFF80EE35003E1F90EE35008E085
:10603000F80EE30602E2F90EE306DECFEEFFF2D73A
:10604000FF0EE3CFDAFFE552FF0EE3CFD9FFE552B3
:106050001200FB0EE3CFF6FFFC0EE3CFF7FFFD0EC1
:10606000E3CFF8FFFE0EE3CFE9FFFF0EE3CFEAFF39
:10607000E9CFF3FFEACFF4FFF90EE35003E1FA0EA4
:10608000E35009E0F90EE30602E2FA0EE306090026
:10609000F5CFEEFFF1D71200FE0EE3CFE9FFFF0EC2
:1060A000E3CFEAFFE9CFF3FFEACFF4FFFB0EE350C3
:1060B00003E1FC0EE35009E0FB0EE30602E2FC0EF6
:0C60C000E306FD0EE350EE6EF1D7120077
:0460CC005B636B5354
:1060D000656E644661696C65645D0A00AAAAAAAA35
:1060E000AAAAAAAA000100000000000102030405F8
:1060F000002077726974696E672043414E206D6598
:1061000073736167650A004572726F72202D0020FB
:10611000696E7374656164206F6620005B536572FD
:1061200069616C436865636B73756D4572726F72FC
:106130003A20005B4672616D65546F6F4C6F6E67FD
:106140005D00506961747461666F726D6120657283
:106150007261746100417676696F206E6F646F20A2
:1061600043414E4C494E200A002876312E30302EC5
:106170003030293A204D61792032352032303036A6
:106180002031323A33333A32370A00417676696F3A
:10619000206E6F646F204D4F4E49544F5220436F15
:0A61A00072736F2043414E200A0085
:0661AA00266AE86A24AE3B
:1061B000E2EF30F0216C221E231E241E2222232215
:1061C0002422261E1FAEEDEF30F01C6C1D1E1E1E7D
:1061D0001F1E1D221E221F22261EF1EC31F01FBEA3
:1061E00004EF31F026AE000C1C6C1D1E1E1E1F1E7F
:1061F000E86A1D221E221F22186C191E1A1E1B1E61
:1062000019221A221B22000C26BEF4EF30F0278838
:10621000FF0C1FC02BF01EC02AF01E502302F4CF2B
:106220001DF0F3CF1CF01F502402F4CF1FF0F3CF6A
:106230001EF02302F3501D26F4501E22E86A1F228E
:106240002A502402F3501D26F4501E22E86A1F2211
:1062500024AE2FEF31F02A501E5E2B501F5A2BAE6A
:0C626000000C23501E5E24501F5A000C3E
:04626C002A0EF66E92
:10627000000EF76E000EF86E00010900F550FA6F7F
:106280000900F550FB6F03E1FA6701D03DD009002A
:10629000F550F56F0900F550F66F0900F550F76FEE
:1062A00009000900F550E96E0900F550EA6E090091
:1062B00009000900F550F86F0900F550F96F090061
:1062C0000900F6CFFCF0F7CFFDF0F8CFFEF0F5C0F7
:1062D000F6FFF6C0F7FFF7C0F8FF0001F85302E140
:1062E000F95307E00900F550EE6EF807F8E2F907F8
:1062F000F9D7FCC0F6FFFDC0F7FFFEC0F8FF0001B4
:0A630000FA07000EFB5BBFD7120086
:06630A001C502102F3CF3C
:1063100018F0F4CF19F02202F3501926000EF420E1
:106320001A6E1C502302F3501A26000EF4201B6E26
:106330001C502402F3501B261D502102F350192635
:10634000F4501A22000E1B221D502202F3501A266E
:10635000F4501B221D502302F3501B261E50210215
:10636000F3501A26F4501B221E502202F3501B2613
:0A6370001F502102F3501B261200FB
:06637A00D9CFE6FFDACFE7
:10638000E6FFE1CFD9FFE2CFDAFFAC6AAB6AFD0EE0
:10639000DBB0AC88DBA202D0AC8CAB8CDBB4AC8EB7
:1063A000DBA602D0AB8801D0AB8ADBA802D0AC84DC
:1063B00001D0AC949E98DBAC02D09D8A01D09D9A0E
:1063C0009E9ADBAE02D09D8801D09D98FB0EDB50DB
:1063D000AF6EAC8AAB8EE552E5CFDAFFE7CFD9FFDF
:0263E0001200A9
:0E63E2001B6A1A6A196A186A200EE76ED890B4
:1063F0001C361D361E361F36183619361A361B3611
:106400002150185C2250195823501A5824501B58F8
:1064100009E32150185E2250195A23501A5A245069
:0A6420001B5A1C2AE72EE4D71200D5
:06642A00D9CFE6FFDACF36
:10643000E6FFE1CFD9FFE2CFDAFFFD0EDB507E0BA6
:10644000B16EB36AB26AA192FD0EDBAE02D0A08239
:1064500001D0A092DBB2CD86DBA002D0B18E01D0FC
:10646000B19EB180E552E5CFDAFFE7CFD9FF120048
:10647000D9CFE6FFDACFE6FFE1CFD9FFE2CFDAFFEF
:10648000E652F00E0001FF17ABAC03D0FF91ABB0AA
:10649000FF81ABB4FF85ABB2FF87AE50DF6EDF503C
:0E64A000E552E552E5CFDAFFE7CFD9FF120053
:0264AE00D9CF44
:1064B000E6FFDACFE6FFE1CFD9FFE2CFDAFFE6521F
:1064C000E652B250DF6E010EB3CFDBFFDECF00F03D
:1064D000DDCF01F000C0F3FF01C0F4FFE552E5524B
:0C64E000E552E5CFDAFFE7CFD9FF12004C
:0464EC00D9CFE6FF1F
:1064F000DACFE6FFE1CFD9FFE2CFDAFF3F0EC716D2
:10650000C66AC56AFD0EDB50C612FC0EDB50C71210
:1065100094869488C68AE552E5CFDAFFE7CFD9FFA3
:02652000120067
:0E652200D9CFE6FFDACFE6FFE1CFD9FFE2CF17
:10653000DAFFFD0EDB50C96EC6AE02D0FF0E03D0EF
:10654000C7B0FED7000EE552E5CFDAFFE7CFD9FF9F
:02655000120037
:0E655200D9CFE6FFDACFE6FFE1CFD9FFE2CFE7
:10656000DAFFACAC04D0AC900001FFB3AC80FD0E00
:10657000DB50AD6EE552E5CFDAFFE7CFD9FF120071
:106580001B6A1A6A100EE76ED8901E361F361A362E
:106590001B3623501A5C24501B5805E323501A5E07
:0C65A00024501B5A1E2AE72EF0D71200D0
:0465AC0015EE00F0F8
:1065B00025EE00F0F86A279C36EC31F08DEC16F0F1
:0465C000FDD71200F1
:0C65C400FF0EE350E84E1200000000D073
:0A65D00000D000D0E82EFAD7120028
:0465DA0000000100BC
:0265DE0000FFBC
:0165E00001B9
:0165E10000B9
:0865E2000000000000000000B1
:020000040030CA
:08000000FFFAFCFEFFFFFAFF0E
:00000001FF
